:020000040000FA
:1000000000F80202FD330000590F00000511000046
:1000100000000000000000000000000000000000E0
:100020000000000000DB000048DB0000590F00006A
:100030000000000000000000590F000065350000BE
:100040004D0D0000590F0000590F00001D34000035
:10005000ED11000049310000E90E0000890F000099
:10006000E50B0000210B0000590F00005D0F0000A0
:10007000C1110000653C00009D330000C933000041
:10008000590F0000590F0000590F0000893500007A
:10009000A9350000590F0000590F0000590F00004A
:1000A000B9390000C33900004F0D0000B132000023
:1000B000590F0000B13100000000000000000000F6
:1000C0000348854600F0FCFC00480047AD73000083
:1000D00000F8020230B50B46014600202022012420
:1000E00009E00D46D5409D4205D31D469540491B6C
:1000F0002546954040191546521E002DF1DC30BDB5
:1001000070B500242546002801DA01244042002968
:1001100001DA01254942FFF7DDFFAC4200D0404241
:10012000002C00D0494270BD03460B439B0703D00F
:1001300009E008C9121F08C0042AFAD203E00B78AC
:100140000370401C491C521EF9D27047D2B201E024
:100150000270401C491EFBD270470022F6E710B522
:1001600013460A4604461946FFF7F0FF204610BD25
:10017000421C0178401C0029FBD1801A7047F8B559
:1001800002464A40D40F42004B0052085B089A4294
:1001900002D20246084611464A0023D0C30D4A0047
:1001A000DDB2120EAD1A202D35DA49020126490AB8
:1001B000F6058A19002C00D0524220214F1B11460F
:1001C000B9402A411018C20D9A4221D0002C17D0F4
:1001D000012D08DCDA05801AD20F8019D207DBB2B4
:1001E00000F0D6FBF8BDDA05801A012340001B069B
:1001F000C01880185A428018CA0F1043490007E0FF
:100200004908C2071143DA05801A8019400880188E
:1002100000F0B6FBF8BD61000122511A001BF7E7A0
:100220000122D2075140AAE70122D2075040A6E797
:10023000024670B54A40D30FDB0740002DD04A007C
:100240002AD0010E140E000212020919400A520AA5
:100250008418E50104465443000A120A2E04504350
:10026000A4194219200CC543AA18120C0125AD038C
:10027000521C521912047F39240400D0521C10431E
:1002800001D44000491EC2B20C06C0092018401C0F
:100290004008802A02D003E0002070BD40084000E2
:1002A000002900DA0020184370BD70B502464A40AC
:1002B000D50F40004A00ED0740085208002814D02E
:1002C000002A12D0C40DD30D41020120C0055202F4
:1002D000490A520AE41A091812187D34914201D3CE
:1002E000641C00E04900002C01DA002070BD0023EE
:1002F000914201D3891A0343400849000028F7D1ED
:1003000000290AD0914202D10121C90705E091429A
:1003100001D2012101E00121C943E005C0184019C3
:1003200000F02EFB70BD0000F0B5074608465840AF
:1003300087B0C00F049048000E4659004008490895
:10034000BC1A884105D2384631461E4617460B4630
:1003500002465800400810434CD0300D0390400531
:100360005900400D490D0590401A0290402872DA5C
:1003700018030121000B090508430190049800921D
:10038000002805D001995242002088410092019036
:10039000029840210A1A0199009800F0BDFA05461A
:1003A0000C466B4607CB00F0D8FAC0197141039A8E
:1003B0000E0D0023D71756401A467A40164344D0F4
:1003C000049A002A2DD0029A012A039A15DC1205FC
:1003D000C01A914101263605001C7141D20F059EBD
:1003E000D2070093019202962A46234600F016FB9C
:1003F00007B0F0BD38463146FAE71605224A0F46E7
:10040000B218C01AB74101210905001C4F4100185C
:100410007F41114618187941E20F10436D1964416C
:1004200013E0E2076D0815436408C2071443039AFA
:1004300001261205C01A91413605001C7141CE07F4
:10044000400830434908C01851412A46234600F06D
:10045000D8FACDE7FFE7049801224000C117121A2D
:1004600000238B4104983146C417381AA141EEE7A6
:1004700030B40124E407634030BC55E730B40124B4
:10048000E407614030BC4FE70000E0FFF0B51FB467
:1004900088B00B990998002448400999C00F490079
:1004A00049080991C0070B990090490049080B9130
:1004B00009990898A64608431CD00B990A98084346
:1004C00018D0099801244000420D4800410D0998B8
:1004D00024050003000B204309900B980003000B38
:1004E00020430B9050181C494018002201901446DC
:1004F000104605E0002001460DB0F0BD032801DAEA
:10050000034600E003239C46C11A0AAE0AE05F00DE
:1005100008ADED5B4F00F75B7D430027AA187C41D7
:10052000491C5B1E6145F2DD410004AB5A522104B7
:10053000120C0A43240C401C0828DFDB01980290AF
:100540000099704601910090059B049A07990698BE
:1005500000F064FAD0E700000DFCFFFFF0B50C4698
:100560005C4085B0E40FE40703944C000026640867
:1005700059009446490802460296224321D0624619
:100580000A431ED06200570D4A000E032303550D87
:10059000012402462C492405781B1B0B360B4018FE
:1005A00023432643614600901C46501AB44103D3AE
:1005B0000098401C009002E0921800985B410028CF
:1005C00003DA0020014605B0F0BD00200121090535
:1005D0000746864611E064461D46141BB54106D306
:1005E0006546521BB341744607430C43A646CD07EC
:1005F00040084908284392185B4105460D43EAD15B
:100600001046184313D060461946504071400843C5
:1006100006D06046101AB34106D20122002306E03C
:1006200000220123DB0702E00122D243531000988D
:1006300074460105381C6141029C039D0019694103
:1006400000F0DFF9BFE70000FD0300000122D20740
:10065000002800DB101A002900DB511A814201D862
:1006600001207047002070470122D207002800DBDC
:10067000101A002900DB511A814201D20120704773
:10068000002070470122D207002800DB101A002941
:1006900000DB511A814201D30120704700207047CE
:1006A0000122D207002800DB101A002900DB511AB2
:1006B000814201D901207047002070470122D207F2
:1006C000002800DB101A002900DB511A814201D1F9
:1006D000012070470020704710B5002904DB0C464C
:1006E0000121C9074042A141002B04DB1C46012324
:1006F000DB075242A341101A8B4101D2012010BDE9
:10070000002010BD10B5002904DB0C460121C907EB
:100710004042A141002B04DB1C460123DB0752426F
:10072000A341801A994101D2012010BD002010BDC3
:10073000C217C10F504010B54018CA0796230021B8
:1007400000F026F910BD10B500229623114600F0E6
:100750001FF910BD0EB5C217C10F5040CA0740188F
:100760000021054B0293019200910A460B4600F0CE
:1007700055F903B000BD0000330400000EB5054973
:100780000291002100910A460B46019100F046F9C2
:1007900003B000BD330400003EB5CA17CB0F0024E0
:1007A00050405140C0186141DA07054B0293019255
:1007B00000942246234600F031F903B030BD00001A
:1007C00033040000C20F410040020123400ADB0550
:1007D000D207090EC0187F2901DA00207047962938
:1007E00003DC9623591AC84001E096398840002A54
:1007F000F4D040427047410040020122400AD20535
:10080000090E80187F2901DA00207047962903DC41
:100810009622511AC84070479639884070470000A8
:1008200070B5CD0F4A0009030123090B1B051943BD
:100830000B4BED070024520D9A4201DA002070BDE7
:10084000074B34339A4203DC9A1A00F075F802E041
:100850000449511888402C43F1D0404270BD00003B
:10086000FF030000CDFBFFFF70B5CD0F4A00090369
:100870000123090B1B0519430D4BED070024520DF5
:100880009A4202DA0020014670BD094B34339A4285
:1008900003DC9A1A00F050F803E0064BD21800F07F
:1008A0003BF82C43F0D0002240428A41114670BDF3
:1008B000FF030000CDFBFFFFC20FD207400040083E
:1008C0000BD0C10D0723DB01C91840020905400AFE
:1008D0001143C2084007114370470020014670478A
:1008E000CB0FDB07490010B5490802460A4307D081
:1008F0000A0D07240903E401090B121B002A01DC7D
:10090000002010BDC900440F0C43C100E018D205FF
:10091000801800F035F810BD10B5202A04DB014620
:10092000203A9140002010BD914020239C1A03469C
:10093000E3401943904010BD10B5202A04DB08465F
:10094000203AD040002110BD0B46D340D040202497
:10095000A21A91400843194610BD10B5202A06DBA3
:10096000CB170846203A1041C1170B4306E00B464F
:100970001341D0402024A21A91400843194610BDCB
:10098000002904DA401C490001D1400840007047AA
:1009900070B40024050C05D11024000402D10029F4
:1009A00021D01124050E01D100020834050F01D118
:1009B0000001241D850F01D18000A41C002801DB4B
:1009C0004000641C002908D020252E1B0D46F54050
:1009D000A14000D001212943084301061B1B000A46
:1009E000DB1D02D5002070BC7047DB05181880188D
:1009F0000029F8DA401C4900F5D170BC40084000DD
:100A0000704710B5002B08DA0024401C6141921891
:100A10005B411A4301D14008400010BDF0B51FB43E
:100A200082B005460C0003D008460BF031F802E016
:100A30000BF02EF820300246009021462846FFF7A2
:100A40006BFF049B059A04460F4618431143084365
:100A500014D0184610431BD0009840210A1A18469B
:100A60000599FFF769FF05460E46009A0599049817
:100A7000FFF752FF084305D0012004E02046394625
:100A800007B0F0BD0020C11705430E432C43374388
:100A900000990E986305401A7905E40A00220C4378
:100AA000FD0A0A3002D500200146E9E701051019C8
:100AB00069410C9C0D9D00196941FFF7A2FFDFE71A
:100AC000064C0125064E05E0E36807CC2B430C3CA1
:100AD00098471034B442F7D3FFF7F6FAC0D50000B8
:100AE000E0D5000030B58C180278401C13071B0FAE
:100AF00001D10378401C120906D10278401C03E0A2
:100B000005780D70401C491C5B1EF9D101E00B708B
:100B1000491C521EFBD1A142E6D3002030BD00008B
:100B200010B52148016A8A0715D44A0715D4C907A8
:100B300032D01E498A89002A15D0531E8B818268C3
:100B40008C6904C48C610A691B040DD0002A22D16F
:100B50000121016010BD022100E00421C1611348A0
:100B60008021416110BD0A69012A09D1026801236F
:100B70009A430260C361FF20683099300C4A1060CC
:100B800001204861CA69002A05D0886909898B005B
:100B9000C01A904710BD10BDFF226832054806A15B
:100BA00009A308F08BFDC04608D00140289501023A
:100BB00080E200E038C500004144435F495251489B
:100BC000616E646C65720000556E65787065637463
:100BD00065642041444320696E7465727275707457
:100BE0000D0A000070B582B00023019344480168EB
:100BF0008A6A4C6813252540132D02D1CB689B07C8
:100C0000DB0F4361930772D453070AD4D30711D182
:100C1000130724D5048F838E1C1B102C0EDD10238C
:100C200010E0042088620220032142A209F0A4FD02
:100C300002B070BD0120886202B070BD048F1B1B22
:100C40001C0610D0DBB20024058FC66A75192D5D15
:100C50000D74641CA342F7D1048FE3180387D206F6
:100C600007D400212FE04B6A0824A3434B62D2062D
:100C7000F7D5CB68C28E448F141B5B04DB0EA342F6
:100C800001D3438FD31ADAB2002A16D0097D438FDD
:100C9000046BE1540199012A10D001231C468901FB
:100CA00045582D7D41184E8F9B19096BCD54641CFE
:100CB000E3B201999A42F2D800E000218B01C318F7
:100CC0005C8FA2185A878A0181184B8FCC8EA34261
:100CD0000BD301230B61805800224262CA6B002AA9
:100CE00003D03A31098801A8904702B070BD0220B4
:100CF0008862044804A1084A08A308F0DFFCC04643
:100D00005490010251C500004145535F495251487A
:100D1000616E646C65720000CE0200004145532094
:100D2000696E707574206F766572666C6F770D0AE8
:100D300000000000414553206F7574707574207574
:100D40006E646572666C6F770D0A000070477047BD
:100D5000F0B589B006205049085EFFF7FBFC04900F
:100D600003914E48406AFFF7A7FD029001910121CF
:100D70004802009000244A4E079107E05948075165
:100D8000069E761C241D642C00D182E030786428F5
:100D9000F7D144480159444F396244480359BB6173
:100DA00043480059B862434A12593A630025591A18
:100DB000059139647B6AF9699941079B00DB2B46F1
:100DC000002B01D0009BC918374F7964FB6A796BFF
:100DD000101A9941079A2F4600DB3A46002A0696D8
:100DE00001D0009A8918FFF7D7FC05460E46324815
:100DF0000059FFF7AFFC029A019BFFF7AFFB0246D9
:100E00000B4638462D49FFF733FB2A463346FFF79A
:100E10003DFBFFF729FD3D46234FB863F963059974
:100E2000401AC10F401840103860FFF793FC244A65
:100E3000244BFFF72BFBB864F964234A234BFFF7DD
:100E400025FB08952A46224BFFF720FB2A46214B1B
:100E5000FFF76AFA05460E4638617961049A039BEA
:100E6000FFF762FAFFF7DCFC074628463146089A8E
:100E7000194BFFF731FC002800D1184F28463146A6
:100E8000089A174BFFF73EFC002800D076E7134F77
:100E900074E709B0F0BDC046F2A201024CBB0000ED
:100EA0002C9701025899010248960102BC9901024F
:100EB00074B40102D8B40102C09801020000F03FEE
:100EC000699006699006903F52257997532ED33F3B
:100ED0000000594000003E40006AF840FFFF020059
:100EE00000408FC098A70102B0B582B0194C2068AD
:100EF000056801A90020087007E090470198401C90
:100F000001A90870C0B2082822D201221104814030
:100F1000294209D02268516080002018826A002A84
:100F2000ECD001A80121E8E7130283402B4201D055
:100F3000022104E082402A42E0D0032113462268C5
:100F40005360800020188268002AD7D001A8D4E717
:100F500002B0B0BD98920102FEE7000010B509484A
:100F60000168CA6920231343CB610269032A08D1AF
:100F7000012293050C689C430C605102C26E0A4327
:100F8000C26610BD08930102F0B581B05C4C2068C8
:100F9000856BE80707D0E168002904D00020884766
:100FA000206801218163A80707D52169002904D0A1
:100FB00001208847206802218163680707D561699D
:100FC000002904D002208847206804218163280773
:100FD00007D5A169002904D003208847206808218B
:100FE0008163E80607D5E169002904D00420884719
:100FF000206810218163A80607D5216A002904D042
:1010000005208847206820218163680607D5616A2A
:10101000002904D0062088472068402181632806E3
:1010200007D5A16A002904D00720884720688021BD
:1010300081630126E80507D5E16A002904D037025B
:101040000820884720688763A80507D5216B0029F9
:1010500004D077020920884720688763680507D590
:10106000616B002904D0B7020A2088472068876393
:10107000280507D5A16B002904D0F7020B2088476B
:1010800020688763E80407D5E16B002904D03703A3
:101090000C20884720688763A80407D5216C0029A5
:1010A00004D077030D20884720688763680407D53C
:1010B000616C002904D0B7030E208847206887633D
:1010C000280407D5A16C002904D0F7030F20884716
:1010D00020688763E80307D5E16C002904D0370452
:1010E0001020884720688763A80307D5216D002951
:1010F00004D07504112088472068856301B0F0BDD5
:101100008893010204217046084204D0EFF309835A
:10111000EFF3088203E0EFF30883EFF309829BB05B
:1011200004A8F0C044464D4656465F4608A8F0C0A5
:101130001846F0C86846F0C018690C902020184482
:101140000D9058690E9098690F90D8691090EFF340
:1011500010801190EFF314801290094908681390E1
:1011600008490868149008490868159007490868F4
:1011700016901793189270461990684608F0B8FCBC
:1011800004ED00E00CED00E010ED00E014ED00E0F7
:1011900080B502F0E1FB0B2005F042F907490A781F
:1011A000002802D0002A05D080BD012AFCD10020F1
:1011B000087080BD0120087080BDC04614900102F7
:1011C00080B5074801210170064802680A430260A1
:1011D00005480268002A02D000200146904780BDE1
:1011E00052A701021C10005054A70102F0B599B09B
:1011F000F548017BC67A427B0E92F44C221F13689D
:10120000F34A1268069242780C9202790592C76AF4
:1012100004931F4001200F907A0200D5BCE03A02EF
:1012200000D5BFE0FA0102D50F98020622605025D2
:1012300008968A191826BB0102D50F984306236029
:101240004123079569430A96354655431426FC0207
:1012500010D50F98040538463746DC4E3460DA4C1A
:10126000A469B464D84CE4697464DA4C241D346015
:101270003E46074690000B90D8040D9068180990E0
:101280000E9B73430F988203B902D04D22D50F985D
:1012900041052960CC480E961646024681692965AB
:1012A000C169696509990D980143089800010818FA
:1012B0000B994018C018C849098892794A43801888
:1012C0000A301C4603F0D2FC234632460E9EC0492B
:1012D00088672A600F98C404380300D52C60F8038F
:1012E00002D50F98000428600F984104B80300D578
:1012F0002960380400D4E4E1039402910E9308922B
:101300000D980B990C180A980C9941430C910F9861
:10131000C0030B90286006F0CBF9002801D003F041
:1013200087FC0C98005B410B43D1099800190E997A
:1013300040180599090140180E90E74D287B079B3E
:101340004343E97A0A010D9C2243D21841188B00CD
:10135000D2180A9B4B43D1186A7B564389190E9EBB
:101360002A791018DF4A128842438818169030688C
:10137000C000800D10A9C882002511957079C007A2
:101380007ED110A80F998182069C00940020E8A2CB
:10139000049B09F0F1F978E00F98820522603A0287
:1013A00000D43FE70F98C2052260FA0100D53BE761
:1013B0003DE7072149030840032149038842089A71
:1013C00000D07EE1069705F04FFE002016900990B0
:1013D0001590C14CE07A217B08180A99414380009E
:1013E0000D9A10434118627B0E9672438A186178F9
:1013F000A379079E7343D718FA683F263240637873
:101400009A420C976ED105960A9A4A4380580F214A
:101410000A0702400398401EC04B1B68DB090340CB
:10142000981810900F98C0020B90B868800767D486
:101430002C46283C08F014F905462068000609D51A
:10144000C3208401786A400704D408F009F9401BDE
:10145000A042F7D905980002B96849080140B3488D
:1014600003688268B868C40C20202040DB0700D0E5
:1014700095E0002310221D461C460E9E0B9FB1E0F6
:1014800010A88582B0681190069C701D924B197946
:10149000E20707D1491C1971D97A1A798A4202D315
:1014A0001D7100E0D97001784278120251188278DB
:1014B0001204891803229143017035715878401C39
:1014C0005870D87A197B08185978884200D85D700E
:1014D000D879401ED871596B002901D010A88847CF
:1014E0007E4DEDE010A80B998182F868304063785A
:1014F000009000207CA20F9909F03EF90E9E94E026
:10150000388A874A024010A8C2822022BA5C930718
:10151000DB0F3C68C3720F9B1A4082726205D20CCB
:101520000D9B1A431692FA68130E0372BB69FC698D
:101530007C4D2D682D0C05745204920F427211934C
:101540001394654CA07B002809980E9E0B9F5FD0DA
:1015500075480068007A0328099859D00C98007DD6
:1015600008400928099853D1C320840108F078F86D
:1015700005460C98406A41070BD459490968090689
:10158000890F06D108F06CF8401BA042F1D90C98E5
:10159000406A41030898884310A9888237E0D2073F
:1015A0000E9E0B9F03D108230022154619E00C9BC9
:1015B0009A68029C224211D19A68520C02249443E8
:1015C0000022134615460DE05CA7010228A000503A
:1015D0003CA10050FC1F000058A701020425002276
:1015E000134614460843104318432843204310A9C8
:1015F000888238420BD10C9B198A494A0A4010A9AB
:10160000CA8219684905C90C0D9A11431691324CCA
:101610002921615C002908D03037B84205D010A9D3
:1016200008461130123107F09DFBE77A2A48047B07
:10163000E519294800790E9027484078401C294632
:10164000FEF748FD88000D9A1043189007996143F2
:101650003801104340182049497B4E4380191C2112
:10166000694340180E9909191B4B1E4A12884A43B8
:1016700080181790099A0C998A60987B002800D0EE
:101680004A629879401C9871187B99798142069F2B
:1016900000D39A715978491C5970D97A0818597829
:1016A00088420E4D00D85A70187A401E18722820B1
:1016B000185C002804D0996B002901D010A8884735
:1016C000089A174202D00F98000328601C4804496A
:1016D000486019B0F0BDC0465CA7010228A00050C8
:1016E0003CA1005058A70102485720455420696486
:1016F0007820256420616E64204554206964782038
:10170000256420696E2052582064657363206D69DA
:10171000736D617463680D0A00000000382000409A
:10172000FF03000094300040F0930102604000404D
:101730004D4143204556542025782025780D0A0038
:10174000FFFFFF03F0B5A5B01E460C9208910024E0
:10175000239422A90C8016A90C8024A909250D80A8
:10176000598C0D91FEF7B6FC2A99012900D0DFE0D3
:101770003189012900D0DBE0318C012900D0D7E08C
:101780000D99002900D1D3E0224607962C990B91A0
:101790002B99069180B205900F9415A805809000B2
:1017A0000E900C990C582E460025204629461746C7
:1017B000FEF74CFF0028119636D12C200A9778436B
:1017C0000899081817A90A4668C868C2E8C8E8C294
:1017D000E8C8E8C2079F119880B280000E5822AD79
:1017E000019523A8009020463946059A069B02F0F1
:1017F0006BFF0F98401C0F90288800282DD03B8A43
:10180000239913AC039416A8029014A8019015AE66
:10181000009617A824AA03F031F925883088119082
:101820000120149E0A9A05E013A8058014952E46FF
:1018300028463A460E9F51000B9B119C5C5259184A
:1018400008830D84D81986600F981885521C0D984E
:1018500082426DD024A805889FE7099616A8002526
:101860000580149524A80688239812902F46109579
:1018700003E06D1CA8B2B04213D8A8B2800017A92B
:101880000C5820461299FEF7EFFE0028F1D1002FE8
:10189000EFD115A8058016A801270780149410948D
:1018A000E7E715A80288B01A012805D115A8068017
:1018B000099F1497119628E010200799095E0129C5
:1018C000119221DB551CA8B20C18109F0E9B099495
:1018D00003E06D1CA8B2844218DDAAB2B242F8D867
:1018E000800017AA10581090394634461E46FEF75D
:1018F000ADFE33462646099C0028EAD115A805808E
:10190000109F14971195E4E7109F0E9B1C463E46CE
:1019100038461299FEF7C9FCFEF754FF0546052824
:1019200000D3052513A8058001200A9A274682E7DF
:1019300025B0F0BDF0B58BB00243159A149C139EF0
:101940002BD0054601A856C0129CD869196A099087
:101950000A911E469F6B0123009309A807AA01461E
:10196000059304F0E3FD716C3846FEF79EFC0746D4
:10197000E06A616BFEF799FC002D069613D00446D1
:1019800011980199012924D10921081A0421069AE4
:10199000515E884229D16425B1E00020308020705A
:1019A00010700BB0F0BDB08800226425002829D04B
:1019B000059269493846FEF773FE0028049C039E91
:1019C0006FD166493846FEF76BFE00281DD05A25B8
:1019D00067E03C25082800D191E05F492046FEF7EA
:1019E0005FFE002819D0502589E00A291DDB1D293A
:1019F0003BDC59493846FEF753FE0022002854D0FC
:101A00005A253AE03346049C39E055493846FEF7FA
:101A100047FE002821D0502543E050492046FEF7DC
:101A20003FFE00282ED0462569E03C25012866D0DF
:101A300049492046FEF734FE0028D4D147492046C4
:101A4000FEF72EFE0028EED145492046FEF728FE7F
:101A5000002854D1434920466EE042493846FEF7FB
:101A60001FFE00281CD128251BE03B493846FEF705
:101A700017FE0022002832D05025049C069B0299B4
:101A8000039E41E036492046FEF70AFE002836D183
:101A900034492046FEF704FE00282FD114252EE0FD
:101AA00037250299059A069B2EE005922B49384668
:101AB000FEF7F6FD002896D129493846FEF7F0FDDD
:101AC0000028B0D127493846FEF7EAFD0028049CDB
:101AD000069B0299039E059A3BD11E2514E00592B0
:101AE0001E493846FEF7DCFD00289CD11C493846CB
:101AF000FEF7D6FD00281DD03C2500E02325049CE0
:101B0000069B0299039E059A25803270002008707A
:101B1000307800280CD118681349FEF7B3FD00286F
:101B200006D12088102803D30F3820800BB0F0BDD9
:101B30000BB0F0BD0B493846FEF7B2FD0028049CFF
:101B4000069B0299039E059A01D11425DCE7232503
:101B5000DAE72D25D8E7C046CDCCCC3DCDCC4C3DE9
:101B6000CDCCCC3C0AD7233C0000204070B588B0D7
:101B70000C4606464088002820D0FEF7E4FD05907C
:101B800005A804A901252A4604F03AFF3088B18847
:101B9000081AFEF7CDFD0390049903A807AA2B4667
:101BA00004F0EEFE5249079D2846FEF779FD002815
:101BB00008D0BF200006206008B070BD0020206063
:101BC00008B070BD4B492846FEF74EFD002804D0F2
:101BD0003F200006206008B070BD47492846FEF748
:101BE0005FFD002801D0002010E000212846FEF70C
:101BF00057FD002801D0022008E040492846FEF7A2
:101C00004FFD002801D0042000E0062001957F212F
:101C1000C905029180003A49091801A806AA0223C1
:101C200004F062FE0698206008B070BDF0B587B081
:101C30000C4605464768002638463146FEF73EFD0D
:101C4000002802D0266007B0F0BD049704A803A9BD
:101C50000126324604F0D4FEA8682968FEF7E0FAAF
:101C60000290039902A806AA334604F089FE20498F
:101C7000069D2846FEF714FD002804D0BF20060666
:101C8000266007B0F0BD1B492846FEF7EDFC002892
:101C900004D03F200606266007B0F0BD164928464E
:101CA000FEF7FEFC002801D0002010E000212846AD
:101CB000FEF7F6FC002801D0022008E00F49284674
:101CC000FEF7EEFC002801D0042000E0062000957D
:101CD0007F21C9050191800009490918684605AAB4
:101CE000022304F001FE059E266007B0F0BDC04649
:101CF000CDCC0C3F295C0FBFCDCC4C3ECDCC4CBEE7
:101D0000F8930102F0B587B00C4606467F2700889D
:101D1000002801D0FD0503E0B08800282ED0334D07
:101D2000FEF711FD03907088FEF70DFD049003A8E7
:101D300002A90126324604F063FE029904A806AA0D
:101D4000334604F01DFE2A49069E3046FEF7A8FCE5
:101D5000002802D03F20010641E026493046FEF728
:101D600083FC002802D0BF20010638E0224930461B
:101D7000FEF796FC002805D0002024E0002020601B
:101D800007B0F0BD1D493046FEF78AFC002801D09F
:101D9000022018E01A493046FEF782FC002801D0E4
:101DA000042010E017493046FEF77AFC002801D0E5
:101DB000062008E014493046FEF772FC002801D0E6
:101DC000082000E00A200096F905019180000F49E3
:101DD0000918684605AA022304F086FD05992846DD
:101DE000FEF726FA206007B0F0BDC046000080BFB5
:101DF000000038433333733F0000C8420000704294
:101E0000000020420000A0410000C04018940102E0
:101E1000F0B59DB015460B917F210391C9051C912A
:101E200002911B9119A900248C801994189417947D
:101E3000598C0691198C0F91DE8B998B07919978AB
:101E400005911F882B21CA432799914201DB7F000E
:101E500015E04022D243914211DC4922D243914203
:101E600002DB7908CF190AE05322D2439142EEDA1D
:101E70005D22D243914201DBBF0000E0FF000A97E0
:101E80001396269E597E00290BD0002132460F461C
:101E9000D170917051701170121D7F1C5C7EA74231
:101EA000F6D30C9311952599149122990D911590C3
:101EB00041088C4211D2FD4A2346A0008458345474
:101EC000270A451C7755250C871CF555240EC01C88
:101ED00034545B1C9CB2A142EFD82398109001208F
:101EE0000990009030463146149A159F3B4604F005
:101EF0002BFB0D9800060890400E139D00D186E044
:101F000068000490002F3FD000221046114614466E
:101F100006E01C461146159F401C82B2BA420ED202
:101F200083B2AB42F8D09200149B9A5E0FB2BA42D1
:101F3000034600DC2346BA42EBDC0A46E9E7002F01
:101F400025D0002210461146129206E01293114647
:101F5000159F401C82B2BA4214D283B2AB42F8D071
:101F6000A5B2AB420CD09200149B9A5E0FB2BA425B
:101F7000034600DC129BBA42139DE7DC0A46E5E704
:101F8000139DE6E7129903E00024214600E00021BA
:101F9000129110980183C4828582049FF057FEF746
:101FA000C7FB7921C9050E91FEF742F91099C86166
:101FB00009980743F057FEF7BBFB0E99FEF738F977
:101FC000109F38622004C40B3057FEF7B1FB0E9906
:101FD000FEF72EF97862601C3056FEF7A9FB0E9CC6
:101FE0002146FEF725F9B86212980004C70BF05796
:101FF000FEF79EFB2146FEF71BF9109CE062781C61
:102000003056FEF795FB0E99FEF712F920631198F2
:1020100005800C98407E410000278D4228463A46B4
:10202000149E1ED30A9880B28AB29300F45E844252
:102030000BDA491C8AB2AA42F6D9002728463A464A
:1020400081B2691A012910D01BE0F018119B198088
:10205000078808040FD0500040008019001F028834
:10206000084681B2691A01290BD1A80030181199CC
:102070000D80078826E00020024681B2691A0129F6
:10208000F3D00A9989B2079B4B43BB421AD30699F6
:102090008A4217D80599002914D0401C82B28918A9
:1020A00003E0401C82B291420CD983B2AB42F8D813
:1020B0009200B35EBCB2A342F3DDB218119B18804C
:1020C0001788EEE712970B980580119800882B1A55
:1020D000002B16DD02210F9A1143032942D10E93E2
:1020E000411C421E10B281420EDA0E98032824DBF6
:1020F0000C98808C012820D019A818A9FFF736FD6C
:102100001FE0002018902BE00026F443374608E03B
:10211000B8B2400019AD2B527F1C521C10B2814244
:10212000E3DB13B2A3423346F2DD159B98423346FC
:10213000EEDA8000149B1B5AEAE719A818A9FFF7EA
:10214000E1FD149E139D0F9A012A13D0032A11D08A
:10215000022A04D111980088281A02280ADA0020DD
:10216000179034E0022A01D1022BB8DA002018902F
:10217000012AEBD1681C691E0FB2B84208DA0C982C
:10218000808C01281DD119A817A9FFF7BBFD1CE001
:102190000022D343144608E0A5B26D0019AF7E5368
:1021A000641C491C0FB2B842E9DB0DB29D421646D1
:1021B000F2DD159DAF421646EEDABD00149E765B49
:1021C000EAE719A817A9FFF7D1FC149E139D249FD5
:1021D000189C17992046FEF723F80F99012900D87B
:1021E000204638600D98002800D1CBE0119908886E
:1021F000109FB8860888281AB880129880B2FEF717
:10220000A2FA7921CC052146FEF712F82146FEF705
:102210000FF8B863119F3888002849D081008919C8
:10222000091F0988129C0C191599884203D2800055
:1022300080198088041915984300534916AA30461E
:1022400004F060FB169810994864FEF7D4FAA4B223
:10225000A04201D14D480FE0001BFEF774FA1C901C
:102260001CA81BA9012204F0CBFB2046FEF76BFA49
:1022700001461B98FDF7DCFF109908603988491B5F
:102280004A1C92B2032A02D20021159F17E009B21C
:102290000229159F12DB3F210906FEF701FA0028EB
:1022A00002990CD10998810709E0C04640210040FD
:1022B0000020129C15998842B9D3BCE73449109884
:1022C00001610898800E5DD0002F1CD000221146BD
:1022D000144610464B1B1DB2ED135B196B40139D4A
:1022E0001BB29200B25E53431818A418491C8AB25C
:1022F000BA42EFD3FEF727FA06462046FEF723FA46
:10230000002C03D100E000260398C0051C901CA8F7
:102310001BA901252A4604F073FB1B9C204631466D
:10232000FDF786FF014610988160002F119422D09E
:1023300000242746264613951291B8B2FEF703FAF9
:102340001299FDF76DFF0546A0001499085EFEF78F
:10235000EFF901461398C00785432846FDF768FF4B
:1023600001463046FDF70BFF06467F1CBCB21598B0
:102370008442E2D300E0002611983146FDF758FF71
:102380001099C8601DB0F0BDF0A00102000020410E
:1023900000004040F0B58FB00692F74A09AF70CA0E
:1023A00070C770CA70C70328079320D88800F3A1AC
:1023B0000858F649FDF7E3FE0446F549FDF7DFFE50
:1023C0000D90F4492046FDF7DAFE0C90F2492046C4
:1023D000FDF7D5FE0B90F1492046FDF7D0FE0A909F
:1023E000EF492046FDF7CBFE0990EE4969E004284D
:1023F00022D0062820D88800EBA10858EE49FDF726
:10240000BEFE0446ED49FDF7BAFE0D90EC492046AC
:10241000FDF7B5FE0C90EB492046FDF7B0FE0B90A2
:10242000E9492046FDF7ABFE0A90E8492046FDF752
:10243000A6FE0990FD4944E00838022821D888000A
:10244000FBA10858D149FDF79AFE0446FC49FDF767
:1024500096FE0D90FB492046FDF791FE0C90FF2063
:1024600081052046FDF78BFE0B90F7492046FDF7CE
:1024700086FE0A90CA492046FDF781FE0990FE4972
:102480001FE08800F1A10858F449FDF778FE0446E2
:10249000F349FDF774FE0D90F2492046FDF76FFEFB
:1024A0000C90F1492046FDF76AFE0B90EF4920465B
:1024B000FDF765FE0A90EE492046FDF760FE0990A3
:1024C000EC4900942046FDF75AFEEC4909680E904D
:1024D000EB480468EB4801684808EB4F05463D406F
:1024E0000022002D08922DD0CA01120E07D0280C10
:1024F000E90D12D14000E649085AE6490AE0C9034D
:10250000090E0CD0280AE90B10D14000E049085A06
:102510008F2189004018E4300DE0DC490AE081B2E7
:102520007F2905D84800DA49085A04E0D94901E072
:102530008F218900401800B2FEF7FAF8D649FDF75E
:1025400077FE02460292039507252606D34B1A68AA
:10255000002A089840D0791C8A420BD21102090E39
:1025600013D0110C1F46D00D1FD14800C849085A7E
:10257000C84907E01F46110E002A13D44800C44979
:10258000085AC2494018E4301FE011041F46090EE2
:102590000ED0110AD00B12D14800BD49085A8F2124
:1025A0008900EFE7BE4808180FE0B84808180CE0AB
:1025B00091B27F2906D84800B549085A05E0B548C8
:1025C000081802E08F218900501800B2FEF7B0F819
:1025D000B149FDF72DFE3B460590159F2C40F50EA9
:1025E0005B69B0491940089810D0DA02D20E34D095
:1025F000C80B3E210140A648405AA6494018E43085
:1026000000B2FEF795F8A449FDF712FE0490149E5F
:102610006800A5A1085EFEF78BF80146A00009AA94
:102620001058FDF7ACFD0146B8B20128089F019192
:1026300002D1022C0AD9A74F052C24D11898089052
:102640000C2D20D80B2D16D3A44918E00027022CFE
:10265000089718D08120C70515E01A04120E00D182
:10266000CAE0080AC90B00D0CDE040008849085AEA
:102670008F218900C2E7092D00D2C7E0964908984A
:10268000FDF77DFD089001200021B542034600D3EF
:102690000B46052C00D308461799169A1A9C199DCB
:1026A0001843069B012B12D1079B402B22D10028F7
:1026B00040D03846FDF763FD01460198FDF75FFD08
:1026C00001460098FDF7ACFD059A04998AE0079B46
:1026D000402B1FD1002838D03846FDF750FD014669
:1026E0000198FDF74CFD01460098FDF799FD059A0C
:1026F000049977E0002833D03846FDF740FD0146C5
:102700000198FDF73CFD01460098FDF789FD059A0B
:10271000049967E000285BD03846FDF730FD01469C
:102720000198FDF72CFD01460098FDF779FD059A0B
:10273000049957E002981146FDF772FD03990029AC
:1027400000D16748059A04994CE002981146FDF7BC
:1027500067FD0399002900D16148059A049941E079
:1027600002981146FDF75CFD0399002900D15C48F1
:10277000059A049936E0C046DCBA0000000068C142
:10278000000088C166665EC1000084C1000084410B
:102790000000B44100004841000020400000F0C0AB
:1027A000000084C10000F841333323C1000050C150
:1027B0009A9929C19A9949C19A9949413333CB4190
:1027C00066667641CDCCAC40333393C09A9949C10B
:1027D00002981146FDF724FD0399002900D14048D5
:1027E000059A049928601046FDF71AFD0899FDF72F
:1027F00017FD20600FB0F0BD99B27F2911D84800B5
:102800002349085AFCE623494018F9E6C12001068D
:102810000898FDF7B4FC0890062D00D933E7002096
:1028200030E78F2189005818EAE6C0463333F34178
:10283000000058C19A9961C19A9969C1000084C188
:102840000000AC4100003841000008C1CDCC80C17F
:10285000CDCC88C133338FC1333397C133339741E4
:10286000CDCC8C413333F3409A9919C0666646C18A
:10287000333397C1CDCCB4410000D4410C000040AB
:102880005030004068400040FFFFFF007C0800001F
:1028900054BE00005C050000919AF63C64200040A4
:1028A0009C0B0000FFFF1F00FAFFFCFFFEFF000073
:1028B00002000400060008000A000C000E001000D0
:1028C00012001400160018001A001C001E00200040
:1028D00022002400000080BF0000A0C0000040C013
:1028E0000000DCC2F0B5FFB0ECB017460E460D900C
:1028F0000021E991E891DC919991989197919691B5
:102900001491139112919AA8F49DF39CF29A002EBF
:1029100000D1E6E10B938030F09B1180099529608E
:102920002546DBAC218095AC21800C952980DA917D
:102930007F24E405B994B894B794B694B594B4944C
:10294000B394B294B194B094AF94AE94AD94AC946B
:10295000AB94AA94A994A894A794A694A594A4949B
:10296000A394A294A194A0949F949E949D949C94CB
:102970009B949A94046644668466C46604674467BC
:102980008467C467046444648464C46404654465FF
:102990008465C465046244628462C46204634463FF
:1029A0008463C463046044608460C46004614461FF
:1029B0008461C461B0090B250B2800D3AE011095CA
:1029C000012B0B9D00D070E12B89012B00D06CE115
:1029D000298C00290E9200D18BE16B8C002B00D149
:1029E000FAE1AA8C3021695C002900D188E10892C3
:1029F000109F5F431196304639460F93FDF76AFBEF
:102A00000590FDF795FE01462046FDF74EFC83211B
:102A1000C905FDF70DFC064696A8021D11988742D0
:102A20000A9200D879E155A811909AA9069196AF1B
:102A300015463A46059C234603F056FF15A80F900D
:102A400006992A46234603F04FFF02230D9338468A
:102A500031463A4603F094FF012308930093E8AA15
:102A600010923846394603F061FDE898DD901198E0
:102A7000069D29463A46234603F036FF0F9829461D
:102A80000A9A234603F030FF384631463A460D9BFA
:102A900003F076FF089B009338463946109A03F0FE
:102AA00045FDE898DE9011982C4629463A46059D4A
:102AB0002B4603F019FF0F9821460A9A2C462B4605
:102AC00003F012FF384631463A460D9B03F058FF9B
:102AD000089B009338463946109A03F027FDE89882
:102AE000DF901198069D29463A46234603F0FCFEE6
:102AF0000F9829460A9A2346254603F0F5FE3846E4
:102B000031463A460D9B03F03BFF089B0093384645
:102B10003946109A03F00AFDE898E0901198069C57
:102B200021463A462B4603F0DFFE0F9821460A9ACB
:102B30002C462B4603F0D8FE384631463A460D9BCC
:102B400003F01EFF089B009338463946109A03F0A5
:102B5000EDFCE898E1901198069D29463A462346F7
:102B600003F0C2FE0F9829460A9A2346254603F031
:102B7000BBFE384631463A460D9B03F001FF089BE9
:102B8000009338463946109A03F0D0FCE898E2905A
:102B90001198069C21463A462B4603F0A5FE0F9855
:102BA00021460A9A2B4603F09FFE384631463A46A4
:102BB0000D9B03F0E5FE089B009338463946109ABA
:102BC00003F0B4FCE898E390119821463A462B466E
:102BD00003F08AFE0F9821460A9A2B462C4603F0F2
:102BE00083FE384631463A460D9B03F0C9FE089BEA
:102BF000009338463946109A03F098FCE898E49020
:102C00001198069D29463A46234603F06DFE0F981B
:102C100029460A9A2546234603F066FE3846314681
:102C20003A460D9B03F0ACFE089B009338463946AC
:102C3000109A03F07BFCE898E5901198069C2146D9
:102C40003A462B4603F050FE0F9821460A9A2B462F
:102C500003F04AFE384631463A460D9B03F090FE9B
:102C6000089B009338463946109A03F05FFCE898B9
:102C7000E690119821463A462B4603F035FE0F9810
:102C800021460A9A2B4603F02FFE384631463A4633
:102C90000D9B03F075FE089B009338463946109A49
:102CA00003F044FCE898E7907AE010880C9A1080D2
:102CB00099919891DA9E08460F46099DF59CFDF77B
:102CC000AFFA2860DC9827606060A6600C34DDA84D
:102CD0000EC80EC42EC82EC42EC82EC47FB06CB031
:102CE000F0BDFF2010800021296020807FB06CB0F3
:102CF000F0BD002201233021695C002900D076E676
:102D0000DDAA1ACF1AC23ACF3AC23ACF3AC20B2141
:102D10003046FDF7DFF9054642E000200690059DAC
:102D20000796089F1190069801460D9C0F9A4A43FA
:102D3000D219109B5A43119BD218D200A358890074
:102D40002E4655AD6B503546121DA25815AB5A5044
:102D5000401C01B28E42E9DC55A89AAE96AC3146D1
:102D600022462B4603F0C0FD15A831460A9A2B4691
:102D700003F0BAFD022320460799224603F000FE25
:102D800001230093E8AA2046214603F0CFFB119BC4
:102D90009800DDA9E89A0A505B1C0B2B1846C1D19C
:102DA000F19EDDA89AA9DCAA0B2303F09DFD092161
:102DB0000E980F9101800B98C168DC9C2046FDF7AE
:102DC00037FA0146A8B2E69F0F281BD808280DD372
:102DD0000846FDF7D4F914E0FF2010800021099A7D
:102DE00011600C9908807FB06CB0F0BD042803D34B
:102DF00081220846D10502E0412208461106FDF76E
:102E000017FA01462B20C04386420D9704DB084683
:102E1000FDF7B5F9014603E04020C043864244DD9A
:102E20000E9A0C9C0B98408A002811D00B98038AAC
:102E300095A80390DBA80290DAA801900094DDA881
:102E40000D4601F01BFE29462488DA9E099D68E0A4
:102E500011910F98208000273D46109705E00E98AD
:102E600004887F1CB8B2A04211D8B8B28000DDA996
:102E70000C5820461199FDF7F7FB0028EFD1002DE3
:102E8000EDD10C98078001250F971094E7E7DBA898
:102E900005800F9A90B2201A012811D10C98048055
:102EA0000D9FDA973E46099D3AE04920C04386428D
:102EB00000DA8BE0FF2208469105FDF7B9F9A9E792
:102EC00010200B990E5E012E00DA90E0551CABB27B
:102ED0001846A1B2AAB28A4217D805E00E990C880A
:102EE000A1B2AAB28A4210D88000DDA90C582046AF
:102EF00010991F46FDF7AAFB3B46002805D10C9808
:102F000005800B98068A0F95109430B2C1186D1C7D
:102F1000A8B28142E2DC109EDA960F9C099D0D9FBB
:102F200011993046FDF7C1F9FDF74CFC052800D397
:102F3000052095A90880A0B20E990988814218D968
:102F4000401C611E0CB2A04218DA12A898A9FEF724
:102F50006DFE0E980188481C491E0CB2A04221DA71
:102F600012A899A9FEF762FE99999898099D0D9F5C
:102F7000A4E600219891999108469FE60022134605
:102F800008E09CB2A40012AF3D515B1C491C0CB27E
:102F9000A042DADB8DB20A2D1546F2D8A400DDADD1
:102FA0002D59EEE70022134608E09CB2A40012AFB0
:102FB0003D515B1C491C0CB2A042D1DB8DB20A2DE5
:102FC0001546F2D8A400DDAD2D59EEE75320C043DD
:102FD000864200DB1BE70E460B9881692046FDF711
:102FE00035FB00280C9C08D10B98808B07E0144619
:102FF000099D0D9F1199109E93E70B98C08BFDF7CB
:10300000A2FB01463046FDF713F9119021E70000BD
:10301000F0B58BB01C4609930E46034600200A907B
:1030200040480088224F05970AA904910394029210
:10303000109C0194012500950B21414389B2303346
:103040001C4A3046FFF74EFC3868079078680890B5
:10305000B868069033480088334F00950194029772
:10306000324E30363249334A3346FEF76BFB069810
:10307000F8620798386308987863099800882E49A1
:1030800005912E4904912E490391029701900096D3
:103090002C4B284629462A46FEF74CFC43200106C5
:1030A0000A98FDF7C5F8FDF78DFB0BB0F0BDC046E3
:1030B000B8A001022CB40102F0B589B00F9F0E9C9C
:1030C000002815D01098079016480088164E012544
:1030D0000095019102960893144B30331449154A18
:1030E000FEF730FB089BF76207983063746303E0D8
:1030F0000D484763C462002518880F4905910F49A0
:1031000004910F490391084902910190074830301A
:10311000009001210B4B28460A46FEF70BFC09B034
:10312000F0BDC0464EA70102F0A80102209A01029C
:1031300010980102FCA70102E89D01024CA70102C0
:10314000F8A6010200A7010280B5124801681F22FB
:103150000A40026003200840022812D10E4802688B
:10316000D30D02D0FF231B06D2180C4B1A600C4A59
:1031700012680C4B1A6080680B4A1080000C0B4AD6
:1031800010801A488268002A02D082680020904786
:1031900080BDC046742000406440004010A8010279
:1031A0007830004014A80102849A0102E6A80102C6
:1031B00080B50D48016889070FD5052101600B48CE
:1031C000C178002908D00021C170C168002903D04E
:1031D000C26841680020904780BD054805A10B4AA0
:1031E0000BA306F06BFAC0462C040040E0930102EA
:1031F000D1C900005048595F54494D45525F49526A
:103200005148616E646C6572000000008D0A000018
:10321000556E657870656374656420696E74657257
:10322000727570740000000070B50446401E0128DD
:1032300014D80320084011D13F2040030818050B83
:10324000281980280AD8164E31780120484029468E
:1032500002F06EFB641E6D1C002CF5D170BDC046E3
:1032600080B50020014602F0ABF8002800D080BDF8
:103270000B480121017080BD70B516460C4605460D
:10328000FF22FCF763FF054831180548027801204A
:1032900050402A46234602F0F3F970BD00E00704CF
:1032A000F0A2010201200003704701204003704793
:1032B000F0B583B030480068C16B0901890F01D0B7
:1032C00003B0F0BDC16BC06B2C4D05404800400FF2
:1032D0000826029686400227384601F017F9019029
:1032E0007043C10B4A1B26485043FCF709FF0446B4
:1032F00006F026F9032123A238461F4F00912346EA
:1033000007F03AFAF88A002817D0019840012946B8
:10331000FCF7E0FE46431822324001200F2A014606
:1033200000D8002173095B181B4CA3420DD8194D1E
:10333000ED1A6D050F2A0CD80CE038680021C16029
:10334000112001F0D3F803B0F0BD5D1C6D050F2A0C
:1033500000D956422A0C029D2E4009018919A34228
:1033600002D80098000400E040040818801839686A
:10337000086303B0F0BDC04670940102FFFF1F0058
:1033800040420F0052434F33324B2070706D202566
:10339000640D0A00FF070000FE7F0000B0B582B098
:1033A000154908688269D2070CD00122C2610D69F3
:1033B000002D07D000686C46214605F0C9FE0021AB
:1033C0002046A84702B0B0BDB0B582B00A4908682F
:1033D000026C92070ED5026C012313430364CD687F
:1033E000002D07D000686C46214605F0B1FE002193
:1033F0002046A84702B0B0BD70940102064801689B
:10340000032291430160016801220A43026000F037
:10341000B5F806F0B7F8C0462800004080B50D4961
:103420000868002810D5224802680423032A01D026
:103430001A4300E01A460A601E490A68002A02D0B0
:1034400041680020904780BD03A00CA19E2211A3DB
:1034500006F034F92C100140696E636C7564652FB9
:10346000647269766572732F6D6B5F736C656570DE
:103470005F74696D65722E6300000000534C454512
:10348000505F54494D45525F49525148616E646CDA
:1034900065720000556E65787065637465642073AD
:1034A0006C65657020696E74657272757074000069
:1034B00008900102ECA80102B0B582B00446007881
:1034C000002811D0094D01A908702868416A002917
:1034D000FCD101A901220020034607F099FE611CDE
:1034E000607800280C46EED102B0B0BD889401028D
:1034F000F0B50C784D782D022C198D78C978090219
:10350000491909040C1981000F4D6C509478D57835
:10351000167852780D4F7B50120292192B021B190C
:103520001B049A180A4B5A50059A13785278094C82
:10353000079D6550084C2468084D6C501102C9184D
:103540004000074A1152F0BD58990102D8B4010257
:10355000BC99010274B4010200970102C0980102F3
:103560002499010280B504480168491C0160006982
:10357000002800D0804780BD58B401020148D549D9
:10358000016070474C90010280B582B00E49086816
:103590000022C2600192CA68002A02D0016801A814
:1035A000904702B080BDC04680B582B00649086928
:1035B0000022C26001220192CA69002A02D0016879
:1035C00001A8904702B080BDE0920102F0B587B03B
:1035D0000120014605F00CF9B548B64903F0AAFBF5
:1035E000B54F387800250028049509D0B3491A3121
:1035F000B34A034610CA0C80891C5B1EFAD14500F1
:10360000B04EB072B88D707179783170B978F17050
:10361000000AB071481CB87030460B30A74C2146E8
:103620004C3105912A46FCF77FFDA8190B30069412
:1036300021461A312A46FCF777FD20207072049843
:10364000787138897070000AB070C320840105F069
:10365000CBF803193B63387881000D3101223046E5
:1036600008F0B8F9B8623E6B05F026F8801905F04D
:10367000D7FC06460C46B548007C05F033FB81B20A
:10368000C90B401800B2C11740103018B86661412C
:10369000F96605F0A9F8B86103F0BEFA0028FBD17D
:1036A0000526304602F0B4FE304602F0C1FE05F0B9
:1036B0009BF8F861386B8449401878630020834A8E
:1036C0000490014608F039F9B86205F08DF8804998
:1036D000B863F9634118481C00D00846386405F007
:1036E00083F83A6C7B4E91197864B9642DE000261A
:1036F000BE7105F079F81E21FCF7ECFC6424601A19
:10370000FDF721F847210906FCF792FD7249FCF705
:10371000CCFDFDF770F805F017FF05F065F80A21FC
:10372000FCF7D8FC601A8949086030463146674A80
:1037300008F003F9B86205F057F8386205F054F85C
:10374000B8613A6C786C634E9119904201D388420B
:1037500071D905F049F8786405F046F8F86103F08E
:103760005BFA00280AD0FDF713FD05F03DF87864F8
:10377000396C8842F3D989198842F0D205F034F8BF
:103780003862B8790228B2D00128DAD10026BE7199
:10379000304631464D4A08F0D0F8B8624F48407A7A
:1037A0002128CED14D494879897909020818B98D67
:1037B0008842C6D17878494909788142C1D14749C0
:1037C0004878897809020818F881397800290AD0E0
:1037D0003A4A4C3200261388834204D0921C761C4D
:1037E000B142F8D10E46F0B238823C6FF96CBA6E35
:1037F0003A4B1E46223600960191029219461A3122
:103800001E331A462346FFF773FE3978388A8842FA
:1038100007D34200294B9A18FB894C269353491C25
:1038200039706421254A115496212C48FCF795FCE7
:103830000020788285E70126304600F037FF3046C9
:1038400008F0A6F8B86EF96EFDF782FA049CFC70D9
:103850003878002828D000241949254608E0069A1F
:10386000521C0692059B9B1C0593091D401E1BD0F4
:10387000069A1378002BF2D05B1E069A1370AE00E6
:10388000DBB22A46164DAB51641C0494FC70530005
:10389000059C2588134CE552074F049C0B68124D7C
:1038A000AB511546551CDAE73C713C7007B0F0BDD2
:1038B00089A90000ED930000B09601022C97010247
:1038C00098A701024EBE0102A06D0100C4090000CC
:1038D000C0C204000026B80300007A4450A80102C8
:1038E00054BD01021CBE0102B8BD010210B582B078
:1038F00008F000F8154C2046143004F0E9FE607919
:1039000007F0FCFD12498A88684682800A88498847
:1039100009048918009103F0A1FE6079052804D0FC
:1039200002220C49092805D003E00122094909288F
:1039300000D0891849792079621D07F0A3FE05F0AF
:10394000E7F9607B05F0E0F902B010BD18900102C4
:10395000F4BA0000889A0102B0B502F047FD154C98
:10396000E060A178002900D0B0BD21790029FBD109
:103970000121217100281AD06425281AA1688142EA
:1039800015D0A0682018007D21698847A068401CD8
:10399000A060A068642801DB0020A060E168A06846
:1039A000022D04D36422511A6D1E8842E9D10020F1
:1039B0002071B0BDD095010280B5002007F0FCF861
:1039C00080BD80B5012007F0F7F880BDB0B582B0AA
:1039D000602833D0622843D0642854D101A82F49ED
:1039E0000180EFF3108072B600242046214601F0DA
:1039F000E7FC2B4D002805D10120020300202946B9
:103A000001F038FC103501AA02232046294602F0B5
:103A10000FF962B623A0FFF74FFD64201B490C523B
:103A200005F028FD1A4800F041FEBFF34F8F1948FA
:103A300019490160BFF34F8F00BFFDE760201349B4
:103A400000220A5205F016FD114800F02FFEBFF3C8
:103A50004F8F104810490160BFF34F8F00BFFDE743
:103A600062200A4900220A520A8005F003FD084834
:103A700000F01CFEBFF34F8F064807490160BFF3FB
:103A80004F8F00BFFDE702B0B0BDC046F2A20102F9
:103A9000A08601000CED00E00400FA05AAAA0000CF
:103AA00000D00204BDF8C8EBC9FDBCB6C4A3CABDB2
:103AB0000D0A0000F0B581B0644FB96808291BD821
:103AC0008A0001A39A589746ED3A0000F93A00009F
:103AD000F93A0000093B0000333B00003F3B000087
:103AE000493B0000173B0000533B0000552848D1DC
:103AF0000120B86001B0F0BDAA2838D1012936D123
:103B00000220B86001B0F0BD0421B9600021B97095
:103B1000787001B0F0BD39797A181073481C38718B
:103B2000C0B27978491F81422FD10820B86001B016
:103B3000F0BD0521B9604649087001B0F0BD06210D
:103B4000B960B87001B0F0BD0721B960387001B03C
:103B5000F0BD797806291AD34B1F002422463D195F
:103B60002D7B521992B2641C9C42F8DB10E00328B2
:103B700007D1022905D10120F8700320B86001B0F7
:103B8000F0BD0020B870B860787001B0F0BD0022C0
:103B9000101841182E4800780918BD7849193C784A
:103BA0000919FA78002A00D0C91CC9B2FF2945D1E9
:103BB000012819D0022841D12748401939460C3133
:103BC0002246FCF7B1FA387B012802D12846FFF7DC
:103BD000FDFE05F04FFCBFF34F8F204820490160E8
:103BE000BFF34F8F00BFFDE71A4EB4710320307151
:103BF000B070AA2070705520307068087071651D13
:103C0000F570400014490918F01D2246FCF78CFAA3
:103C1000301DE11CEAB2D21C037892B2D218401CCB
:103C2000491EF9D1A019D143C171090A01720934A1
:103C3000002031462246034607F0EAFA0020B87019
:103C4000B8603871787001B0F0BDC046609501026F
:103C500050900102AA970102F2A201020CED00E0CD
:103C60000400FA0580B582B0002001900448C268C3
:103C7000002A02D001A80021904702B080BDC046B2
:103C800018950102F0B583B000242046FFF7E8FA4A
:103C9000FFF70BFB274EB060FFF704FB7060264F69
:103CA0000BE001A8C1888088084319D101A8408889
:103CB00024180834B068844235D201AD0821284662
:103CC0002246FFF7D9FA28880028EAD0B8422AD03D
:103CD00001AD0421284600F0D3FCA9888842E5D034
:103CE0003460B06884420CD201AD022128462246DD
:103CF000FFF7C2FA2888B84203D0A41CB0688442F7
:103D0000F2D370682118491E4042084030600DD03F
:103D10000024254601202946FFF786FA03CE4D19D7
:103D2000083E8542F6D3346003B0F0BD0024346011
:103D300003B0F0BDA0960102FFFF0000F0B585B012
:103D40001F4604920646C8170C1844400A2C0391DB
:103D500014D301250A212046FCF7BCF96D1C632C05
:103D60000446F7D804998D4200D329460A9C002FB7
:103D700009D00398002808D4002207E001250499FF
:103D80008D42F2D2F2E7002205E001220423234013
:103D90009B081343FA1A0223234004980028029434
:103DA00012D1002B10D0F468002C62D403980028A4
:103DB00025D40298400734D57068B5686F1C8742D7
:103DC0002FD830682B2423E0E407ECD1002A0AD155
:103DD000E9E7376820203855B560F068441CF46086
:103DE000521E002CDFD49142DDD27768B468651C86
:103DF000BD42EED9F468521E002CF4D5D3E7404200
:103E000003907068B5686F1C87420AD830682D240B
:103E10004455B760F068441CF4600025ED43A842A7
:103E200027DB002B1CD00120029B1840049B184369
:103E300016D1002A03D113E0521E002C0ED4914259
:103E40000CD27068B3685D1C8542F5D830683024A8
:103E5000C454B560F068441CF460EDE7002C08D44D
:103E60000092029801900A2230460399049B00F0C8
:103E700003F805B0F0BD0000F0B587B01F46154649
:103E80000290012406919142009407D301240698E0
:103E90002946FCF71FF9641CA842F9D20D980C9A28
:103EA000BC42039700D3039400990140002A00917B
:103EB00009D00029029C25D12021800705D408467D
:103EC000002F11D004E0029C1CE03020002F0BD00A
:103ED000084609E023685854A260E168491CE16083
:103EE0003246721E00290DD4039991420AD2164619
:103EF0006368A1684A1C9A42ECD9E1683246721E96
:103F00000029F1D5E068002859D40590012401E08A
:103F10007F1E6C43022FFBD2069821461646FCF703
:103F2000D9F83246A842F4D2029880680490069FDD
:103F30000195069738462146FCF7CCF8049D691C8C
:103F4000029F7A68914206D9069F059A019D0592C3
:103F5000002A0ED516E01B4A125C3B685A55B96020
:103F6000FA68521CFA600491069F019D0592002A8E
:103F700008D460433F1A20462946FCF7ABF8AC4210
:103F80000446D6D200980028029C059B049D16D0BA
:103F9000002E14D0701C01E0002B10D4401E039999
:103FA00081420CD2691C62689142F5D822682023B4
:103FB0005355A160E268531CE3600D46ECE707B07F
:103FC000F0BDC0468CBD000070B5002801D00120B6
:103FD00070BD0C461625284600F090FA284605F0DC
:103FE000A9F8002C05D01B48183014222146FCF7F4
:103FF0009BF828211748415C002915D04168002909
:1040000016D403220B469343144A9C588D07ED0E99
:10401000FF26AE40B4439C501F220A40012191402C
:104020000F4A11600F4A116001210161002070BD2B
:104030008A07D20EFF2393400F220A40083A032139
:104040008A43054954589C43545001210161002082
:1040500070BDC046549001021CED00E000E400E099
:1040600080E200E000E100E05A21014A505270472E
:10407000209A01025C21B4480022425282847A21B3
:1040800041840284C2830283C28202821149416058
:104090008260C2603D21490441834182090C8183D1
:1040A000818270475C21A8480022425282847A2192
:1040B00041840284C2830283C28202820549416034
:1040C0008260C2603D21490441834182090C8183A1
:1040D000818270474C37373770B59C484C2101605E
:1040E00001252C02601C00F089F9322000F0DEFA74
:1040F00000F072F9284600F079F9284600F088F8B7
:1041000000F064F90C4800F079F900263046314699
:1041100000F084FA2846314600F080FA204600F08C
:104120006DF9022000F06AF94834204605F03EFAA5
:1041300005F09CFA70BDC0460102000010B50446AF
:10414000072106F075F907480460032406A22046FB
:10415000214606F011FB0AA20F4B2046214606F02D
:104160000BFB10BD9896010248656C6C6F2066725F
:104170006F6D204D4B53454D49210D0A0000000045
:104180004275696C6420696E666F726D6174696FE7
:104190006E2025730D0A000048DB000070B5042472
:1041A00000252046294602F073F9012620463146B3
:1041B0002A4602F045F905222046314602F090F9E0
:1041C00070BDB0B505200424214602F061F9062532
:1041D0002846214602F05CF90A20294602F058F9E7
:1041E0000920294602F054F900240121204602F05A
:1041F0004FF902212046224602F072F9B0BD0000BC
:104200000248016801229143016070475800004054
:1042100002490A6802408242FBD1704704600040B4
:10422000B0B5494D28688107484C0ED528797F21C3
:10423000084022688A431018206023680B4002203F
:104240000321434A06F098FA286880040ED55E20C0
:10425000285C7F21084062688A43101860606368A8
:104260000B40022003213B4A06F086FA172000F09B
:1042700045F93948016802220A4301218A43026054
:1042800036483749016037480021C17181791F25BF
:1042900029408171817A427C837C1B029A18C37CFD
:1042A0001B04D218037D1B06D2182F4B9A4218D13B
:1042B000427B837B1B029A18C37B1B04D218037CAE
:1042C0001B06D218294B9A420BD1C27A037B491E96
:1042D000122906D819028918254A914201D12021B4
:1042E00001720178CA0602D11022114301701C3CF0
:1042F00020682021884320601E481F4901604168D2
:104300000029FCD503F01AF90446022003211BA260
:10431000234606F031FA0A20C441032C05D80220B6
:1043200003211DA206F028FAFEE71848C1680F22F3
:104330009143C1600168164A0A40026019200001D9
:10434000144948600D60B0BD889A010248000040E1
:1043500080C500006AC50000040200400C06004051
:10436000AF6B100A6B0001404D383650312E32369B
:104370000734000000600040FE1C00804368697044
:104380002049443A20253038780D0A00C8600040A2
:10439000FEFFC3FF0C0400404F6C6420636869702B
:1043A000206D6F64656C206973206E6F7420737567
:1043B00070706F727465642062792074686973200C
:1043C00053444B2121210D0A0000000080B5172025
:1043D00000F08CF8002080BD10B51724204600F0B6
:1043E0008DF8204604F0A6FE002010BD0121C9076B
:1043F00001430148016070470060004010B5C1B240
:10440000000AC2B202290CD0012913D0002930D1F0
:10441000911E7F4802291BD20121032A2AD0490478
:1044200029E07B484168002A1FD00246203A114308
:10443000416010BD76480168D31E022B10D3012ABB
:1044400029D0002A41D1012292079143016010BD79
:10445000002A16D10121490702688A43026010BD73
:104460000123042A1FD05A041EE00122920791431F
:10447000416010BD0904194A7F32C36A13405918BC
:10448000C16217498A699207FCD501214907026870
:104490000A43026010BD0522120791430246203AEA
:1044A0000A43026010BD1A04836A0C4C1C40A21817
:1044B00082620B4A131F00241C600A4B0A4C1C60CA
:1044C0000D235B0214681C431460054A93695B0664
:1044D000FCD5052212071143016010BD80FFFCFFCF
:1044E0001402004004010040FF0F00000121814040
:1044F000474802688A4302607047C04601218140F4
:10450000434802680A4302607047C04610B5052858
:1045100011D8C0467844007940008744020E19241F
:1045200034393B490A680868C0003CD53A4820390C
:104530000A425DD03BE0002010BD35490A6808689A
:10454000C00035D534480B46203B1A4237D134E001
:104550002F490A680868C00036D52F480B46203B13
:104560001A424CD135E02A494C680120C0030A6840
:104570000B46203B1C421AD00C68E4003BD5264C6D
:104580001A423CD03AE0224800680120C00310BD26
:104590001F490A680868C0001ED51F480B46203B0B
:1045A0001A4220D11DE01B4820390A4220D010BDFC
:1045B00018480B46203B1A4201D10120C00349682C
:1045C0008900890FC84010BD12480B46203B1A4293
:1045D00015D10120C00312E00E480B46203B1A42C1
:1045E00001D10120C00349680903890FC84010BDEB
:1045F0000120C00310BD074C1A4200D020464A6873
:104600009200920FD04049680901890FC84010BD3F
:1046100020000040006CDC020026B80304282CD8DF
:10462000164AC0467844007940008744020A121AAC
:1046300021000320000713688343880780081818A7
:104640001AE00320800613688343880700091818BE
:1046500012E003208004136883438807000B1818B6
:104660000AE0FF200002136883430802181803E0E1
:104670001068FF23984340181060704724000040E2
:10468000B0B5002200290CD0074B047895B22D0A52
:1046900065406C001C5B12026240491E401C0029F0
:1046A000F3D190B2B0BDC0468CBB000000280AD048
:1046B00030B407252C02CD25641960434009123817
:1046C000001FFDD830BC7047F0B583B01F461646BA
:1046D0000D460146E8680291FBF7AAFD04460F2E3D
:1046E00011D8082E04D320462146FBF748FD09E0E7
:1046F000042E02D38120C10501E04120010620469D
:10470000FBF796FD04460999089E2B20C04387427B
:1047100005DB20460F462146FBF731FD0DE03F202B
:10472000C04387420BDA4920C04387420CDBFF209D
:104730000F4681052046FBF77BFD39460446688A13
:104740000880346003B0F0BD01915320C04387421C
:1047500006DB20462146FBF712FD0446688A10E07E
:10476000A8690299FBF78EFF002801D1A88B00E011
:10477000E88BFBF7E8FF01462046FBF759FD0446AE
:10478000002001990880346003B0F0BDF0B581B01D
:1047900005460120072D66D80C46002963D04A4FF4
:1047A00038680169C90736D105263046FFF7A6FEED
:1047B000304604F0BFFC03CF0369012213430361B9
:1047C000002918D403200B4683438E481E588807BF
:1047D000C00EFF278740BE434027874037438948A4
:1047E0001F501F20084082408748026087480260AF
:1047F000354800680FE08A07D20EFF2696400F2347
:104800000B40083B03218B437D495F58B74340264B
:1048100096403E435E50690140180121090242184A
:10482000E369DB069B0CA569ED00EDB2EB18536064
:1048300062685207520B23685B075B099A18A368EA
:104840005B079B0CD218E3685B075B0DD2182369EA
:104850005B01DBB2D21863699B07DB0ED2188023A1
:1048600013434350002001B0F0BDC046F0B581B005
:10487000002A23D005460835134C2668F668EE401A
:10488000F50702D0022001B0F0BD069D8600A619F2
:10489000B560400124682018009301231D024619C9
:1048A00077680724A7437760F16032610099B160AF
:1048B000415919434151002001B0F0BD03A00AA1A4
:1048C00074220DA304F0FAFE98920102696E636CE3
:1048D0007564652F647269766572732F6D6B5F64A2
:1048E0006D612E6300000000646D615F7472616E23
:1048F0007366657200000000496E76616C69642021
:104900007472616E7366657220647374206164648E
:104910007200000000015849085840687047C046BE
:10492000F0B581B005460120012D4CD80C46002978
:1049300049D0002D03D0012D04D10F2000E00E201E
:10494000FFF7DCFDA668012E04D0002E4FD1E089D0
:1049500000284CD12901294843580020D860F50788
:10496000AD0F27686668B607360F76192569EA071E
:10497000920EB618022F04D0012F03D10122164344
:1049800000E040361D4F9E60E2681A6079188D6025
:104990006269CA604968002917D403220B46934311
:1049A000184A9C588D07ED0EFF26AE40B443802672
:1049B000AE4026439E501F220A4001219140124AD8
:1049C0001160124A116001B0F0BD8A07D20EFF24B7
:1049D00094400F230B40083B03218B4308495D584B
:1049E000A543802494402C435C5001B0F0BD08A046
:1049F0000FA1492212A304F061FEC046E092010219
:104A00001CED00E000E400E080E200E000E100E0F6
:104A1000696E636C7564652F647269766572732F55
:104A20006D6B5F6475616C5F74696D65722E630098
:104A30006475616C5F74696D65725F6F70656E003F
:104A4000636F6E66696720697320696E76616C6951
:104A5000640000000001084A10580160816880224B
:104A60000A4382607047C0460001034908588168C4
:104A70008022914381607047E0920102F0B58DB0D1
:104A8000019315460E460A9012980024089004805F
:104A9000149F3C801398099004601598049004803A
:104AA000FF2081053046FBF7C3FB0290304603969A
:104AB0003146FBF764FB2B463D460690274607959B
:104AC0000B9311E01180188880002858099908601C
:104AD0000120079D28800520049908807F1CBCB216
:104AE0001888844200D9A0E028880028F6D1A000C8
:104AF0000A9D2E5830460699FBF7B6FD002817D0C0
:104B000030460399FBF7B0FD00280B9B079DE5D1CC
:104B1000089A1780099D2E601888011B012934D13D
:104B20001080198889000A9A51582960059035E04B
:104B3000089A1780099806600B9B1988081B0128A2
:104B4000C0D00C96019825187E1CB0B28542BFD308
:104B500089B2B2B28A420ED880000A990C58204617
:104B60000C99FBF773FD0B9B002804D10998046096
:104B7000089806800C94761CB0B28542A8D3198898
:104B800089B2B2B28A42E7D9F5E70C960199621868
:104B90007D1CA9B216468A4205972CD2059884B28C
:104BA000A5000A9E7259002C104609D0A819001FB2
:104BB000016810460C92FBF7E2FA0C9A062C07D813
:104BC0000446A81941681046FBF7D9FA0C90204614
:104BD000079D0299FBF756FD00280B9B07D10C9807
:104BE0000299FBF741FD0B9B002800D076E70120DE
:104BF0002880032070E780B2AAB282420FD88800D2
:104C00000A990C5820460C99FBF720FD0B9B0028B5
:104C100005D1099804600898058005950C946D1CD1
:104C2000A9B28E42BAD31888E5E70DB0F0BD0000F6
:104C30000A490A680A4802400A60FD214900094AF7
:104C40001268515C002908D007490A6C02400A64C6
:104C5000012000060A6882430A6070470004004091
:104C6000FFFFFF7FF093010220000040002070470B
:104C7000F0B583B00D4604467C264643504887195C
:104C8000F869396AFBF726FAA84200D892E0019544
:104C900002940121EFF31080084002D1EFF310825B
:104CA00072B63C4610343B690025062B0CD80A46E8
:104CB0009A40D3065B0F06D161231A4275D00D4688
:104CC000002803D003E00225002800D162B6002DA1
:104CD00002D0284603B0F0BD00943C46203438484A
:104CE00080591021C1613E46143604F0B9FC0546D6
:104CF0003868C069C00605D504F0B2FC401B318895
:104D00008842F5D90621029D284600F00BFF206855
:104D100001994143B86909183868816017217956AB
:104D20003C461734002909D5C16920220A43C261D3
:104D30000121F966890502680A43026005212846B7
:104D400000F0F0FE207840B200250028C1D42B48A6
:104D500000687D24E100FBF7BDF961014143029841
:104D600000F0B2FE04F07CFC04463868C069C0075D
:104D700005D004F075FC001B31888842F5D904F099
:104D80006FFC04463868C169890706D504F068FCE1
:104D9000001B31888842F5D938680121009A1160DA
:104DA00053498161284603B0F0BD032121600028EA
:104DB0008CD08CE7034804A1084A09A304F07EFCC8
:104DC00008930102B0C50000666C6173685F626C95
:104DD0006F636B5F65726173650000005D020000C8
:104DE000626C6F636B20696478206973206F7665ED
:104DF000722072616E67650D0A0000006CB40102DA
:104E0000F0B583B002907C214143934A5418E56E7B
:104E1000EAB2511E02291FD229040126090E18D018
:104E200001960092022100F07DFE2746143704F01F
:104E300017FC06462068C169890606D404F010FCF8
:104E4000801B39888842F5D92068007DC007019E03
:104E500008D0304603B0F0BD032A36D100922804B2
:104E6000000E36D020466C302D0C002101910160DF
:104E70002746143704F0F4FB06462068C069C007D3
:104E800005D004F0EDFB801B39888842F5D904F089
:104E9000E7FB06462068C169890706D504F0E0FBF8
:104EA000801B39888842F5D9206811498161E9B2AF
:104EB0000120002911D003290099019E00D006206D
:104EC0002061226F002A0ED1C3E70026304603B0CE
:104ED000F0BD0126304603B0F0BD0099019E20616F
:104EE000226F002AB5D002A89047304603B0F0BD2B
:104EF000000093EB70B5002801D0012070BD78252B
:104F0000CD4E705D00280ED000240921204600F00F
:104F100009FE0F20FFF7CAFB1520FFF7E7FA7455CB
:104F20003461204670BD042070BDC046F0B581B02C
:104F30000C460078484EF16881422CD1032C54D1A4
:104F4000706EB16E884261D900240621204600F0BF
:104F5000E9FD3068F16D81602046214600F0E2FDF8
:104F6000354660352CCDF0683168B48C414F0097E0
:104F70005B1BA34200D81C46A3081431FFF776FC44
:104F8000B06E0019B066306E00193066F06D001911
:104F9000F06501B0F0BDB168814255D1032C45D117
:104FA000F08CF16D0918F165316E09183166B16E3A
:104FB0000818B066716E814238D900240621204657
:104FC00000F0B0FD3068F16D81600121204600F0F5
:104FD000A9FD316EB068F38C3268264C009414320F
:104FE0009B08FFF743FC01B0F0BD30681021C161A0
:104FF00004F036FB05463068C069C00616D504F0DB
:105000002FFB401BB18A8842F5D90FE03068102190
:10501000C16104F025FB05463068C069C00605D5AE
:1050200004F01EFB401BB18A8842F5D90120C1075C
:10503000326813688B431360F16E22040A43000246
:105040001043F06601B0F0BD4D200201034804A1F9
:10505000844B04F033FBC04608930102B0C5000046
:10506000666C6173685F646D615F63616C6C6261E3
:10507000636B00002D4F0000F0B581B000786E4DDD
:10508000AA68824200D0D0E001263002032942D132
:105090006A6DAA66AB6DAC6AA418EB652C66AB6C46
:1050A0005B1CAB646B6E934235D95E30FFF7FEFA42
:1050B000686CA96C02293AD3814238D1E88C696DB9
:1050C000081868650020062100F02CFD2868E96DAD
:1050D00081602F6D04F0C4FA04462868C069C007D7
:1050E00005D004F0BDFA001BA98A8842F5D904F066
:1050F000B7FA04462A68D069800706D504F0B0FAEA
:10510000001BA98A8842F5D92A687420285C0128E6
:1051100041D0F10440E0F2072B681C6894431C6006
:10512000EA6E090411430143E96601B0F0BD0229AA
:10513000FBD38142F9D2E88C696D09186965A96DC4
:105140000818A8650020062100F0ECFC2868E96D2D
:105150008160EF8C04F084FA04462868C069C007B7
:1051600005D004F07DFA001BA98A8842F5D904F025
:1051700077FA04462A68D069800706D504F070FAE9
:10518000001BA98A8842F5D92A687420285C012866
:1051900022D0F10421E03105334B3B40591801285E
:1051A00002D01920400601E00720C00608182F4948
:1051B00040185060002F0DD004F052FA04462A68BF
:1051C000D069800706D404F04BFA001BA98A8842F4
:1051D000F5D92A682B6D1FE03105234B3B40C918D8
:1051E000012802D01920400601E00720C006081857
:1051F0001E4940185060002F0DD004F031FA0446CB
:105200002A68D069800706D404F02AFA001BA98A0C
:105210008842F5D92A68EB8C296EA868144C009452
:105220001432FFF723FB01B0F0BD044804A10C4A7F
:105230000C4B04F043FAC04608930102B0C50000CD
:10524000666C6173685F646D615F77726974655FD6
:105250006E62797465735F63616C6C6261636B002D
:105260007204000097C50000FF3F0000008080002E
:1052700079500000F0B587B004460126880E14D09E
:105280001546002A11D00F468120C004401B8842D9
:105290000BD37C206043F04908180590818C384678
:1052A0000691FAF717FF002902D0304607B0F0BD8B
:1052B00028460699FAF70EFF0029F6D1059880696D
:1052C0003E1A30460699FAF705FF0746039670190D
:1052D0000190069E3146FAF7FDFE0546C01B04907C
:1052E0000598006A02903146FAF7F4FE049981426B
:1052F0000FD20026BD42D8D92046394600F018FB0F
:105300002046FFF77DFD0028FAD17F1CAF42F3D382
:10531000CBE700900398029D2946FAF7DBFE06468C
:10532000284670430399081A019800D0761C294634
:10533000009D7543FAF7CEFE05900299414301980E
:10534000401A03900699FAF7C5FE0490AF420BD2BB
:105350002046394600F0ECFA2046FFF751FD0028C0
:10536000FAD17F1CAF42F3D305988642069D009F79
:105370000CD220463146FFF77BFC2046FFF740FD6C
:105380000028FAD1761C05988642F2D30398A842E9
:1053900003D20026304607B0F0BD059847430025EC
:1053A000E919204600F0C4FA2046FFF729FD00283D
:1053B000FAD16D1C002604988542F1D375E7C046EA
:1053C000F0B585B0002803D00124204605B0F0BD1B
:1053D0007822A14FB85C002803D00024204605B0F5
:1053E000F0BD0492002905D0384614300CC90CC019
:1053F0001CC91CC00020F86615242046FFF77EF863
:10540000204603F097FE38681021C16104F028F9A6
:1054100004463868C169C90607D504F021F9001BA4
:10542000B98A8842F5D9386800E0B98ABA7D12078E
:10543000120B5218F97DCB07DB08D2188B07DB0F54
:105440005B05D218CB06DB0FDB05D2184B07DB0F51
:10545000DB06D2188B06DB0F5B07D2180907C90FD2
:1054600089071143016000240A21204600F05AFBFD
:105470003220FFF71BF90821204600F053FB04F00F
:10548000EFF805463868C169890606D404F0E8F8E3
:10549000401BB98A8842F5D93868017D0A46C23A6C
:1054A0005342534174257B550904027D1202511861
:1054B000007D0B180220032668A2314605F05CF936
:1054C000785D0128039619D1F87D02900026062107
:1054D000304600F027FB0721304600F023FB012176
:1054E00002988143785D012847D1386889010175A8
:1054F00006757521795C012938D048E00020032128
:1055000000F010FB04F0ACF806463868C169890663
:1055100006D404F0A5F8801BB98A8842F5D938680A
:10552000007D46080122F87D014631431640C90737
:1055300001D0304036D00295002506212846019240
:1055400000F0F0FA07210095284600F0EBFA0198E8
:1055500046400298385C012813D13868B1010175C2
:10556000009901757521795C012910D114307621DB
:10557000795C4A424A41510008E0386806754900A2
:1055800003E03868009901757100143001703748E4
:1055900000687D21C900FAF79DFD282141430020C4
:1055A00000F092FA7720385C012803D10220002114
:1055B000FFF734F804F054F806463868C069C007AD
:1055C00005D004F04DF8801BB98A8842F5D904F063
:1055D00047F806463868C169890706D504F040F8DF
:1055E000801BB98A8842F5D93868D0498161172073
:1055F0003856002829D57868002816D40146039A21
:1056000091431C4A8B588507ED0EFF26AE40B343ED
:105610008026AE401E438E501F210140012088404D
:1056200015490860154908600FE08107C90EFF227F
:105630008A400F230340083B039883430C481D58BE
:10564000954380228A402A431A50012004997854B5
:105650003861204605B0F0BD089301026A656465B3
:10566000635F69642025780D0A0000006CB40102B4
:105670001CED00E000E400E080E200E000E100E07A
:10568000F0B593B07C270A9047439348C619980712
:1056900004D0F07D4024044000D017E10125880E9D
:1056A0002ED0002B2CD08120C004C01A884227D3D2
:1056B00009920122EFF31084144002D1EFF310801D
:1056C00072B63046103005903069002506280891E2
:1056D000069310D8079414468440E106490F04D17C
:1056E00061210C4203D0154604E0022502E00221AC
:1056F000059B1960079C002C00D162B6002D02D0DA
:10570000284613B0F0BD344617347348C0591021F1
:105710000491C1613746143703F0A2FF0546306893
:10572000C069C00605D503F09BFF401B398888423D
:10573000F5D92078400665D40297B78C069C2046A0
:105740003946FAF7C7FC079039464143601A03907F
:1057500035462435A74200D894E0039800281CD091
:1057600006210A9C204600F0DDF928880799484365
:10577000089940183168886000272046039C394604
:1057800000F0D0F9079B099A28885843C01931685E
:10579000097D11547F1CA742F6D330680499C1617A
:1057A00003F05EFF0446029D3068C069C00605D55F
:1057B00003F056FF001B29888842F5D903F050FFFB
:1057C00004463068C069C00705D003F049FF001BDC
:1057D00029888842F5D903F043FF04463068C1693F
:1057E000890706D503F03CFF001B29888842F5D9BC
:1057F00030680121059A1160B2498161002528466F
:1058000013B0F0BD03200025089FF76509993166A4
:1058100006997166B566F0660120C00731680A68AE
:1058200002430A6006210A9C204600F07BF930689A
:1058300087602046294600F075F93A4F0BAA0A9274
:105840001BCF1BC21BCF1BC2B48CF0680A99FEF79A
:105850009DFFF0683168344A0092069A944200D362
:105860001446A3081431099AFFF700F8B06E001926
:10587000B066306E00193066F06D0019F06528468C
:1058800013B0F0BD002404E0641C0798844200D3E8
:1058900063E706210A9800F045F9288860430899D3
:1058A00040183168886000270A98394600F03AF9B4
:1058B00028880028099AE7D0604310183168097DCC
:1058C000C1557F1C28888742F6D3DDE7034804A131
:1058D000064A07A303F0F2FE08930102B0C50000D8
:1058E000666C6173685F726561640000C6030000E6
:1058F00054686520444D412072656164206C656E7A
:105900006774682073686F756C64206265207468C2
:1059100065206D756C7469706C65206F6620340D40
:105920000A0000000CBE00002D4F0000000093EBA9
:10593000F0B583B00D4604467C264643514887198E
:10594000F869B98CFAF7C6FBA84200D894E0019533
:1059500002940121EFF31080084002D1EFF310828E
:1059600072B63C4610343B690025062B0CD80A461B
:105970009A40D3065B0F06D161231A4277D00D46B9
:10598000002803D003E00225002800D162B6002DD4
:1059900002D0284603B0F0BD00943C462434394878
:1059A00080591021C1613E46143603F059FE054668
:1059B0003868C069C00605D503F052FE401B318827
:1059C0008842F5D90621029D284600F0ABF82088D0
:1059D00001994143B86909183868816017217956DF
:1059E0003C461734002909D5C16920220A43C26107
:1059F0000121F966890502680A43026004212846EC
:105A000000F090F8207840B22C4600250028C0D441
:105A10002B4800687D21C900FAF75CFB20492D3135
:105A20004143204600F050F803F01AFE044638685F
:105A3000C069C00705D003F013FE001B31888842FF
:105A4000F5D903F00DFE04463868C169890706D50B
:105A500003F006FE001B31888842F5D93868012121
:105A6000009A116017498161284603B0F0BD0321F7
:105A7000216000288AD08AE7034804A1084A09A3C4
:105A800003F01CFE08930102B0C50000666C617350
:105A9000685F736563746F725F6572617365000040
:105AA0002B020000736563746F722069647820694B
:105AB00073206F7665722072616E67650D0A000053
:105AC0006CB40102000093EBF0B583B001917C222D
:105AD0000290424353498C182546143503F0C0FD0B
:105AE00006460221029800F01DF803F0B9FD0746B2
:105AF0002068C169890606D403F0B2FDC01B29885D
:105B00008842F5D92068007DC00708D06420FEF7E0
:105B1000CDFD03F0A5FD801B01998842E1D903B0BA
:105B2000F0BDC046F0B585B0049104467C206043CA
:105B30003C490F183D46143503F092FD064638687F
:105B4000C069C00705D003F08BFD801B29888842FF
:105B5000F5D903F085FD06463868C069800705D58C
:105B600003F07EFD801B29888842F5D91421049B0F
:105B70005943DC2060432C4A1018039002914018CE
:105B8000018A8268C47C7426BE5D012E0DD101910C
:105B9000012B02990CD0012B0DD07526BE5D012E74
:105BA0000ED0019E072B0ED10EE00E4602990BE09F
:105BB0000222012BF1D138247526BE5D012EF0D1D1
:105BC0000326072B00D0019E184B33402406920772
:105BD000D20A1219D218039B5958C907490C5218F6
:105BE0004168CB071B0CD218837C5B075B0BD21878
:105BF000C0684007000A10183A685060002E0ED0A6
:105C000001290CD103F02CFD04463868C0698007D7
:105C100005D403F025FD001B29888842F5D905B07D
:105C2000F0BDC0460893010254BF0000FF3F0000D2
:105C3000F0B59DB00D460126890E2FD0002B2DD03A
:105C400011928121C9041093C91AA94226D30121B6
:105C5000EFF310840C4002D1EFF3108272B67C2275
:105C60000F904243E74814928718384610303B693A
:105C70000026062B0DD80A469A40D3065B0F07D1A3
:105C800061231A4200D16FE30E46002C03D003E0DB
:105C90000226002C00D162B6002E02D030461DB084
:105CA000F0BD0290BD650021139179651098401EEA
:105CB00012904019B964B9690D916E1A1199B962BF
:105CC000FD6238637E63F98C0E913046FAF702FA72
:105CD0000446B863129830180E9E3146FAF7FAF966
:105CE000109B011B4A1CF86339647A64139A0029DB
:105CF000194608D0704359190D9BC91A0A1A7443E2
:105D0000581B80190119384648300E9038464430E7
:105D10000D90384640300B90384626300590384676
:105D200058301390384654301290F9643A651498FC
:105D3000B44908581021C1613846143014903846CF
:105D4000503004903D464C3503F08AFC04463868D8
:105D5000C069C00606D503F083FC001B14990988AE
:105D60008842F4D9F87D40060C9500D574E20123F1
:105D70000E9803600D98016800290F9800D1CDE2BC
:105D80003A4674320A92DA0407921A0509921922E5
:105D9000520606920722D206089216E09A48006838
:105DA0007D21C900FAF796F9109941430F9C2046CE
:105DB000FFF78AFE20460C9D0E9A11684B1C13605B
:105DC0000D9909688B4200D9A8E20B9A1268012A42
:105DD00055D0002A00D0A8E02E6812990C681399BB
:105DE0000D6806211091FFF79DFE386885601198B7
:105DF000051903F035FC04463868C069C00706D0B1
:105E000003F02EFC001B149909888842F4D903F092
:105E100027FC04463868C169890707D503F020FCD0
:105E2000001B149909888842F4D938680A990A78BD
:105E3000012A089900D00699012A099A00D0079AE8
:105E40003346724C234013430B4371490B43436069
:105E5000002EA3D003F004FC04463868C069800714
:105E600006D403F0FDFB001B149909888842F4D97D
:105E70003868297801756D1C761EFAD18EE7012BE2
:105E800000D0C7E02E6812990C6813990D6806219E
:105E90001091FFF747FE386885601198051903F0E7
:105EA000DFFB04463868C069C00706D003F0D8FBA2
:105EB000001B149909888842F4D903F0D1FB0446E9
:105EC0003868C169890707D503F0CAFB001B14991C
:105ED00009888842F4D938680A990A78012A089909
:105EE00000D00699012A099A00D0079A3346474CF8
:105EF000234013430B4346490B434360002E69D0B4
:105F000003F0AEFB04463868C069800706D403F08E
:105F1000A7FB001B149909888842F4D938682978AE
:105F200001756D1C761EFAD154E0012B00D0C9E03A
:105F30002E6812990C6813990D6806211091FFF7CD
:105F4000F1FD386885601198051903F089FB044656
:105F50003868C069C00706D003F082FB001B1499A3
:105F600009888842F4D903F07BFB04463868C1698C
:105F7000890707D503F074FB001B14990988884230
:105F8000F4D938680A990A78012A089900D0069944
:105F9000012A099A00D0079A33461C4C2340134328
:105FA0000B431B490B434360002E13D003F058FBF7
:105FB00004463868C069800706D403F051FB001B13
:105FC000149909888842F4D93868297801756D1CBC
:105FD000761EFAD10C4800687D21C900FAF77AF8DC
:105FE000109941430F9C2046FFF76EFD20460C9D03
:105FF0002A68139B196889181960129B19688918F7
:106000001960D9E6089301026CB40102FF3F000059
:10601000008080008B4200D0CEE604990E68129971
:106020000C6813990D6806211091FFF77BFD386805
:1060300085601198051903F013FB04463868C069A0
:10604000C00706D003F00CFB001B14990988884296
:10605000F4D903F005FB04463868C169890707D500
:1060600003F0FEFA001B149909888842F4D93868B5
:106070000A990A78012A089900D00699012A099AF2
:1060800000D0079A3346D44C234013430B43D349E3
:106090000B434360002E00D180E603F0E1FA044692
:1060A0003868C069800706D403F0DAFA001B149937
:1060B00009888842F4D93868297801756D1C761EE4
:1060C000FAD16BE6129A1268119CA618139A1568F9
:1060D0008B425FD104990C6806210391FFF722FDE2
:1060E0003868856003F0BCFA05463868C069C007A7
:1060F00006D003F0B5FA401B149909888842F4D9F8
:1061000003F0AEFA10900C9D3868C169890708D574
:1061100003F0A6FA1099401A149909888842F3D915
:1061200038680A990A78012A089900D006991091CE
:10613000012A099A00D0079A2346A7490B40134326
:1061400010990B43A5490B434360002C14D003F076
:1061500087FA10903868C069800707D403F080FA86
:106160001099401A149909888842F3D9386831780F
:106170000175761C641EFAD19A4800687D21C90019
:10618000F9F7A8FF039941430F9C2046FFF79CFCB9
:10619000204611E605990C8806210391FFF7C2FC01
:1061A0003868856003F05CFA05463868C069C00746
:1061B00006D003F055FA401B149909888842F4D997
:1061C00003F04EFA10900C9D3868C169890708D514
:1061D00003F046FA1099401A149909888842F3D9B5
:1061E00038680A990A78012A089900D0069910910E
:1061F000012A099A00D0079A234677490B40134396
:1062000010990B4375490B434360002C14D003F0E5
:1062100027FA10903868C069800707D403F020FA85
:106220001099401A149909888842F3D9386831784E
:106230000175761C641EFAD16A4800687D21C90088
:10624000F9F748FF039941430F9C2046FFF73CFCB8
:10625000204605990A88CCE65E4815A90A4678C802
:1062600078C278C878C20125E8073A681368034302
:106270001360B868FEF78AFA02200026139C216892
:10628000BA6AF9653A6610997966BE66F8660C983E
:106290000068129A1168091811600E9B19684A1C4F
:1062A0001A60226810182060002900D0F6E41095CA
:1062B0003846603013903C465C34384608301290C3
:1062C00006210F98FFF72EFC3868216881600C9832
:1062D0000068119003F0C4F904463868C069C0072B
:1062E00006D003F0BDF9001B149909888842F4D93F
:1062F00003F0B6F90446109D3A68D069800707D5C7
:1063000003F0AEF9001B149909888842F4D93A6861
:106310007420385C01282DD0E9042CE003F0A0F9AA
:1063200004463868C069C00706D003F099F9001B1D
:10633000149909888842F4D903F092F90446386820
:10634000C169890707D503F08BF9001B14990988E7
:106350008842F4D938680121029A1160224981618A
:10636000002630461DB0F0BD04210160002C00D194
:1063700091E491E42905119C174B234059180128F9
:106380000C9D02D01920400601E00720C006081825
:10639000124940185060002C0ED003F061F90446F9
:1063A0003A68D069800707D403F05AF9001B1499A2
:1063B00009888842F4D93A682B68139801681298C2
:1063C0000068074C00941432FEF750FA30461DB0B6
:1063D000F0BDC046CCBD0000FF3F00000080800043
:1063E000795000006CB40102000093EB3120C00032
:1063F00001490968085870479892010210B50124B4
:106400002046FEF77BF8204602F094FE002010BDE7
:10641000012181401C48006842688A4342607047FD
:10642000194909680968C140012008407047C04601
:10643000012181401448006842680A434260704765
:10644000012907D0002910D1012181400F4802689D
:106450000A430FE0012181400B4800684368002A8D
:106460000DD00B4343600161704701218140074813
:1064700002688A43026004480068416170478B43A8
:10648000436001617047C0468893010208010040E3
:10649000124A072809D880000F2383408140194001
:1064A000106898430843106070470F280AD880008E
:1064B00020380F2383408140194050689843084397
:1064C00050607047800040380F238340814019405E
:1064D00090689843084390607047C046340000407D
:1064E000F0B54307DC0E0726A640C3089D000E4BFF
:1064F000EF187D68B5433E1D002908D035600122A4
:10650000824001290CD1186810431860F0BD0121A8
:106510008140186888431860A24015433560F0BD7B
:10652000186890431860F0BD0C01004010B582B0AF
:1065300014460A4601460498009301900820234619
:1065400000F092F802B010BDB0B584B014460A460F
:1065500001460898022500950193029007202346E2
:1065600000F052F904B0B0BD70B500285BD03149DD
:106570000A783149002A03D14A68012313434B604A
:10658000428803881B049A180B46183B1A608288BD
:1065900083891B049B180C460C3C23600B46083B6C
:1065A00084681C60446903232340057CAD00EB181C
:1065B0008569AD072D0D5B19457C2D035B19C569F8
:1065C000AE07B60A9B19867CB6059B190E1F336071
:1065D000036A122B04D107240C60541EA2410AE066
:1065E000032C05D1012D03D807220A60012202E005
:1065F00006220A600122114C002525700F24640137
:106600002034C57C6D0225401B069B0BD218C37934
:106610001B07DB0ED21880790007C00D1018401937
:106620001439086070BD064806A1862209A303F04C
:1066300045F8C04650A701021810005052A70102A9
:106640008EC800006C73705F656E67696E655F72FF
:10665000756E0000506172616D65746572206973BA
:10666000206E756C6C000000F0B58BB0109E340489
:106670003ED00D46D64C2140012701977F06B942F6
:106680003CD111462140B9423FD11C40BC4243D1CC
:10669000119902AC0027E781E78066802780278276
:1066A000A774E1749908A181A908A1800A900997AB
:1066B00008970797900880B204902046FFF754FF90
:1066C000AA480078002801D00BB0F0BDAB480168A3
:1066D000C90708D10168C90705D10168C90702D1F6
:1066E0000168C907F3D07F48019901700BB0F0BD74
:1066F000B8480D49AF22C14B02F0E0FF0095B54804
:106700000949B022754B02F0D9FF0092B148064901
:10671000B122724B02F0D2FF0093AE480249B2227E
:106720006E4B02F0CBFFC04664C80000F0B58DB0E0
:106730000392139E340446D00A46A54C21400125FD
:1067400002956F06B94244D103992140B94247D11D
:106750001C40BC424CD11499129D04ACE1742949EF
:1067600021820027E781E780668027809908A18140
:106770009108A1800B95012D01D16121CF43A77410
:106780000C9002200A9009900398800880B206902D
:106790002046FFF7E9FE75480078002801D00DB0CB
:1067A000F0BD76480168C90708D10168C90705D15D
:1067B0000168C90702D10168C907F3D049480299A5
:1067C00001700DB0F0BD83480D49FB228B4B02F0E8
:1067D00075FF00927F480A49FC22404B02F06EFF91
:1067E000039800907B480649FD223C4B02F066FF6F
:1067F000009378480249FE22384B02F05FFFC04602
:1068000071C800008E8E0000F0B58BB0119E34046C
:1068100047D00D466E4C2140012701977F06B942B3
:1068200045D111462140B94248D11C40BC424CD10F
:106830001299109F02ACE174294921820021E18163
:10684000E180668021809908A181A908A18009972B
:10685000012F01D0712100E06121C943A1740A9088
:10686000032008900790900880B204902046FFF71C
:106870007BFE3E480078002801D00BB0F0BD3F48B9
:106880000168C90708D10168C90705D10168C907AE
:1068900002D10168C907F3D01248019901700BB009
:1068A000F0BD4C480C49D522544B02F007FF00952F
:1068B00048480949D622094B02F000FF009245489A
:1068C0000549D722054B02F0F9FE009341480249E1
:1068D000D822024B02F0F2FE80C80000AEC80000D1
:1068E0008686000052A7010210B582B014460A46FF
:1068F000014600200093019004202346FFF7B4FED8
:1069000002B010BD10B584B014460A4601460020FE
:1069100000900193029004202346FFF707FF04B084
:1069200010BD000070B50D46064604242046FDF754
:10693000E5FD204602F0FEFB0B4805600B480670A3
:10694000002E0ED00A48016880220A437F218A4324
:1069500002600120000307490860074908600748F2
:106960000460002070BDC04654A7010250A7010278
:106970000CE400E080E200E000E100E01C100050C8
:10698000B0B582B0144602461148204001256D067C
:10699000A8420DD1180413D01748016000200093BD
:1069A0000190062011462346FFF75EFE02B0B0BDFF
:1069B0000094FF228C320748074908A302F07EFEAC
:1069C000FF208C30421C034803490C4B02F076FE3A
:1069D0000300FCFF8EC8000056C8000044737420FA
:1069E0006164647265737320257820697320696E11
:1069F00076616C696400000008100050CCC800008B
:106A000080B582B00B460146002000920190032021
:106A10000A46FFF729FE02B080BD0000002801D021
:106A2000042100E00221C54A5172411E88418001C3
:106A300003490A6840239A43101808607047C0460B
:106A400050A00050F0B583B002912E49CD7A0E7B54
:106A5000771987424FD90899019118254543412656
:106A6000F604BF00BE19745B34490C4057033C194F
:106A70009B07D90C6418324B1B681B7A7453751929
:106A80006C880326B60326409B079B0C9B193F246A
:106A900004401819029CA3061B0DC0186880012A27
:106AA000184E13D8707B14224243307B502343434B
:106AB00024011B199A18F37AC0181C234343D018D9
:106AC00080081E4A104007430F432F8001986860DA
:106AD00001F08AFEA860E8681A4908403030E86092
:106AE000286908402721715C4018286100F0DCFD0E
:106AF000686103B0F0BDFF228832034803A108A3F8
:106B000002F0DCFD5CA701021DC900006D61635F3E
:106B100063735F636F6E737472756374000000005B
:106B2000435320696E646578206973206F766572BF
:106B30002072616E67650D0A00000000FF0700000B
:106B4000F09301020000F0FF2820D84900220A54E7
:106B50007047C046F0B581B0009314460D46074615
:106B600006263046FDF7CAFC304602F0E3FA26213D
:106B70001D4847540021017041708171017181707D
:106B80004171C170C17102224272C16201634163ED
:106B9000816304734273C572009A561C134A1680AF
:106BA00001724120C00401214903F9F7D6FA5020AF
:106BB00060432901081861198A00801818224A4385
:106BC0008018B2B24A4380180949401809498842DE
:106BD00004D200F0B5F8002001B0F0BD064807A1CE
:106BE0009A2209A302F06AFD5CA7010258A70102DC
:106BF00028000802012008021DC900006D61635FC2
:106C0000696E697400000000454D206F76657266FC
:106C10006C6F770D0A000000A448C179002901D0EB
:106C200001207047007A411E88417047F0B583B05B
:106C300002912A494B7B834248D9CB7A0C7BE318DB
:106C400018245C439B00E3184124E4041A1914241B
:106C50000190054665430026565100925519EE886D
:106C60002E4F0B467A1C3240F54E3688497A711AFF
:106C70002B4E0E40B618EE803740997BEF80AA88E5
:106C8000284F17404A424A4191007918264A8918EC
:106C9000A980264F0F402D1D029801280AD12449B2
:106CA0000E400921C902711869800121C9037918B0
:106CB000298000E02F800198444300980019074A7A
:106CC000918C4182118C018203B0F0BD3520C2004D
:106CD000034804A109A302F0F1FCC0465CA701022D
:106CE0001DC900006D61635F6C696E6B5F646573E5
:106CF000635F636F6E737472756374004C696E6B5F
:106D0000206465736320696E646578206973206F01
:106D10007665722072616E67650D0A00FFFBFFFFEA
:106D2000FF03000003D0FFFFE80F0000EF1F00008B
:106D3000FF830000BE4A5063916370475CA7010265
:106D4000F0B581B04348CC21016003214160B849CE
:106D50000A7BD304404C1B19CC7AA218541E1C4346
:106D60001823534392009A184B7B14255D43521904
:106D7000920122430124630613434361002282628D
:106D8000C262026342638263C26342650267334B3D
:106D90001A605A609A60324B1A601A619A61DC611B
:106DA000304C1C62304C251D1D6325460C3D5D6337
:106DB0002546283D9D632D4EDE631C645C642C4D8E
:106DC0002F461C379F642746143FDF64103C1C6528
:106DD000284C5C65284C9C650C369E67274CA56347
:106DE0004035E563DA651A665A669A66DA661A67A6
:106DF000234DDD6702258561224DC561C325AD03A5
:106E0000CD620A63D2435A601F4A1368FF25AB4321
:106E100026254D5DAD072D0EEB1813601B4A102380
:106E200013601B4A1360272260238B541949816029
:106E3000C160016121607D21090101664166164939
:106E4000C164164941641649016400F01DFC01B09B
:106E5000F0BDC04604A000500000F8FF94A0005010
:106E600034A10050FF185A003004004004100040C4
:106E70001C2000405430004060400040B8A1005049
:106E800014001400FF3F3FFF04E400E080E200E054
:106E900000E100E0DC05DC053F0270020133D007B1
:106EA000D007D0072921C64A505470475CA7010279
:106EB000F0B58BB0079208910146C14FB87809919F
:106EC000FFF7B4FE78793A7B79790691824200D84F
:106ED0009FE0FB7A9A181823534392004124E1045F
:106EE00004915218D2187B7B14214B43D2185024A2
:106EF0006043155801230A93DB022E469E43165029
:106F00004E4B2B4005937D7B03914D433E7B744359
:106F1000F97A0B011B195B1971181C240294614347
:106F20005918A84B1B88069C5C430919C904490DD4
:106F3000059BC91811501018079941603878797964
:106F4000089A00920322099BFFF77CFDF87A397BAF
:106F500009183878814263D983000993049AD45C74
:106F60000894F7212140D154D1184D788E783602FB
:106F70007619CB781B04F31807900A9886051E43F0
:106F8000330CCB70FB7A387BBC784D709F4D35400D
:106F9000039E6643C018029B4343981940029C4BD2
:106FA00003405C19200A8870200CC870F023089DEB
:106FB0002B401B1D3D7B0895FE7A099D5355C870DB
:106FC0000620079A50438019089A801848701F229B
:106FD000D20222400243100A88707879401C7871EE
:106FE000387B7979814201D3002179713978491C44
:106FF0003970F97A08183978884201D80020387039
:1070000028200A993954387A401C3872387A0BB0E3
:10701000F0BDA7204200D2480649074B02F04EFBC4
:10702000A72042007A32CE487349744B02F046FBE7
:107030005CA701023DC90000E6C8000000F0FFFFA8
:1070400058A701020320000605490A6882430A6026
:107050000A6802430A600348012101607047C04684
:107060001C0000401CA0005080B50120FDF7FCFC76
:1070700080BD0000F0B587B006930646504C607A9C
:10708000504B1B88181A0C9DA84200DC89E00F4663
:107090000592012E06D156480021C1620169554A68
:1070A00089180160A0783146FFF7C0FDE078E178EB
:1070B000069A2B4600F0AEF82078E178009700227F
:1070C00006923346FFF7BEFCE07A217B0818217850
:1070D00088426ED94120C20404918800815C0391EA
:1070E000F7250D40029285544549455C4549465C6B
:1070F000360276194449475C3F04F6190127BF055B
:1071000037433E0C4654E67A217BA3783C4A8554AB
:107110003E4D3D4014275F4389191C234B43D91929
:1071200049023B4B0B405D19290A364BC1542E0CCA
:1071300035494654F02703990F400599002900D19D
:107140003F1D217BE37A029A87542F4A86540622F8
:10715000049E7243D2185118294A81541F22D20228
:1071600015400D43290A274A8154E078401CE070FD
:10717000E07AE178814201D30699E1702178491CD7
:107180002170217B08182178884201D80698207048
:10719000E079401CE071A07A401CA072E07907B051
:1071A000F0BD3920C2001632074808A109A302F039
:1071B00085FA3920C20004480F49104B02F07EFACC
:1071C0005CA7010258A701021DC900006D61635F41
:1071D000747800004D4143205458206C656E20693E
:1071E00073206F7665722072616E67650D0A00000C
:1071F0000804004090D0030053C9000004C90000F7
:10720000010008020200080203000802FF07C0FF95
:1072100000F83F00F0B589B00893019204914F4DFA
:10722000EF7A874200D891E0297B502632464A43C4
:107230004124E3040693D218CC19A1005118182256
:10724000059254430A19697B142307935943531831
:1072500002900001195804460390504A0A40A97A46
:10726000C902511808988205D2088A181A514C4947
:1072700011402A7B00965643384CE57A2C0106983B
:107280002418A719354E5419A5007D1905984443B3
:107290002819747B079D6C430519049FD219414836
:1072A000048854432A19089CD204520D51181D46D3
:1072B0000398195000F002FA0146707A001902048E
:1072C0003E460CD080B2C000002900D1801E029F33
:1072D000A5214900F8F7FEFE1F21014001E0002131
:1072E000029F38012818427983791B029A18C379C2
:1072F0001B04D2182C4B1340437109045918090C74
:10730000C171002C20D0154835460646007B009BF5
:107310004343F17A0A01069F3A43D21841188B0081
:10732000D218059B4B43D118727B079B5343C91856
:1073300040191C4A1288424388180199884203D098
:1073400001992246F8F7F0FE09B0F0BDFF225C3249
:10735000034804A109A302F0B1F9C0465CA70102E9
:107360001DC900006D61635F74785F646573635F5E
:10737000636F6E7374727563740000005458204418
:1073800045534320696E646578206973206F766584
:10739000722072616E67650D0A000000FF0700E051
:1073A00000F8FFFF58A70102EFFFE00082B0FCF7F2
:1073B00093FE052000242146FFF76AF806202146A7
:1073C000FFF766F80A202146FFF762F809202146F8
:1073D000FFF75EF80125284603F0F6FA204603F091
:1073E000F3FAFCF7EEFE2046FCF7A8FE01F022FEC1
:1073F00001F01AFE4348016843480068890308D435
:107400000321090708402907884202D0FCF732FE11
:1074100006E0FCF737FCFCF745FE0020FDF76AFDAF
:10742000FCF7FEFE0024204604F0FEFAFEF7E6FF1D
:10743000FCF7B4FE35483649016000F093F8724E0F
:10744000B088344D2880FF2006307080B07A3249F1
:1074500008707D20C000F188F8F73CFE2F490870C5
:107460002B6803252E4A2846294603F085F97088A3
:10747000C1B20091030A2B4A2846294603F07CF941
:1074800029496422294B204603F09CFD01F086FB2C
:10749000FCF72CFA0125264A2846294602F024F852
:1074A000244802F051F8244F7878002815D07C70D9
:1074B00004263046FEF7BCFFFCF788F83046FEF79E
:1074C000A7FFFCF749FA0B20FEF7AAFF397800283E
:1074D0000FD00029E8D13D70E6E7FCF73DFA0B201C
:1074E000FEF79EFF3978002807D00029DCD13D70D7
:1074F000DAE70129D8D13C70D6E70129D4D13C7014
:10750000D2E7C0461800004030000140E09501027B
:10751000B53A0000DC960102B196010270B4010296
:1075200047C800002AC80000E4950102F9B1000034
:10753000C1940000CC0C00001490010201480068C6
:107540007047C0460C00004081B080B581B0039305
:1075500003AB009302F088FD01B080BC02BC01B017
:1075600008470000F0B581B0002630463146FDF7EF
:1075700027FF0125AC022349234F30463A462346D4
:10758000FEF77EF839882148814238D064217E5246
:1075900062217E5260217E5244217E5250217E52D1
:1075A000FD87BD8778217987022139874321F986B4
:1075B000BE83FD811649B9817E810A213981154931
:1075C000B9803880FE831420B8827D208000F88046
:1075D000EFF3108072B630463146FDF7F1FE002819
:1075E0000CD12A0300263046064D2946FDF742FEFF
:1075F000054A304629462346FEF71AFB62B601B01B
:10760000F0BDC04600E00204F2A20102AA5500004B
:10761000E1FF0000341200000020704710B5002484
:10762000002809D0002905D003464A00034819461E
:10763000F8F77AFD204610BDE04310BD009301022B
:10764000014600200A2901DAC0437047014A11802F
:107650007047C046849301020020704780B50188BE
:10766000064A11808178064A1170C178054A117066
:107670000079FCF7F9FC002080BDC046DC930102D4
:10768000DE9301020CA8010204480549016015219E
:1076900009044160034981607047C0469C30004046
:1076A000410008003400070007480068406970473F
:1076B000FD20400004490968085C704702480068E2
:1076C0006221405C7047C046F093010210B5064845
:1076D0000468064800686421F8F712FD0221C943D6
:1076E0004143081910BDC04610A8010214A80102A8
:1076F0000A491A220A600A4948704878FF2109029B
:10770000084A13688B43800380B2C0181060064893
:107710002021016005480160002070477020004072
:10772000E093010204E400E080E200E000E100E018
:10773000F0B5A9B016460F460546C648002B0246CE
:1077400000D01A463921CC003D21C90051181191B1
:107750008242189206D001204202BE491898F8F7DA
:10776000E3FC189A6120111913910E21119C0A91C2
:10777000A170002F0D9501D00A2100E009215923A5
:1077800017938300E170784278411399087030783C
:1077900010901070F17AE17471785170B778977029
:1077A000F178D1703579157174795471B17991711D
:1077B000F179D171317A1172717A5172B17A917213
:1077C0007E1EF0B200210328169106D870B2800008
:1077D000A1A210586A00805A169017988200189833
:1077E000C0181490F81E022804D3012E084604D8AD
:1077F0009D4800E09D48031918781290189DA8181C
:1078000017902846303015902C4656346D20800055
:107810002950974A974B149E33627262B362F262A8
:107820003176F182139B597009229A7028184160B1
:107830008160C1600161109880008F490858F9F794
:107840003BF8012F10900F9104D0022F05D17F211A
:107850007E2004E07C217B2001E05B215A20159DE5
:10786000A984207003200C90A080012666701F2040
:107870000B90A8821820A8740A46083A179BDA765B
:10788000169B129AD2184A439100189A9163B70234
:10789000791E8B420E9109D9784860803420688423
:1078A0007748288277481399088339E07F2B10DDC9
:1078B000802B18D031028B421BD071028B4227D112
:1078C0006E49618068846F4813990883CF20C00097
:1078D00025E0202B17D0402B1AD168486080042067
:1078E000688469481BE065486080062068846748B2
:1078F00015E062486080102068846248139908830C
:10790000C520C0000BE0624860800220688404E06B
:1079100004206884812040006080FF20023028829B
:10792000104600F005FF1298102806D0402808D114
:1079300008201499C876072000E004201799887061
:1079400002E017980C9981701898169A8078C11ED9
:1079500002290CD3022811D001280CD12672BA4278
:1079600000D900266672BA4213D8F44812E00D20FE
:107970000002119908800120800201E00C980002A9
:107980002081BA4201D8EE4800E0FA2017998860B9
:107990000EE0FA2017998860139800780028119952
:1079A00001D0E8484880E848139A1083E7480880E7
:1079B000A88CF8F7E3FE0026E54B3246F8F766FDA3
:1079C00002460B46E3493046F8F7C8FDE24B324623
:1079D000F8F75CFDF8F724FF0746E080DF49304602
:1079E000109A0F9BF8F7BAFDDD4B3246F8F74EFDC3
:1079F000F8F716FF78434042800B608116990E9885
:107A0000814208D90C20149FB872D64817998883F0
:107A10001220189A0EE0480A189A149F01D00D20DF
:107A200003E0080A00D1DBE20A98B872CE48179941
:107A300088831220F872D078052844D878440079D9
:107A4000400087440227402C3339C848B881C848D1
:107A50002FE0C046989001029CBD00009CBD000034
:107A6000ACBD0000ACBD0000FABA000001BB0000D4
:107A700030750000102700004CBB0000050200001C
:107A8000FF060000040800000A040000360400009D
:107A900003020000B748F881B748388013E0B748C0
:107AA000F881B7483882B74838600CE0B448B881EC
:107AB000B5481799C88306E0B4487882B448B880BE
:107AC0000B9800069064AE483881A748F880B1480A
:107AD00002882A84B0480078E874B0480078119F82
:107AE0007875387D139000285ED0AD490A68102360
:107AF000DA413A600A794B79CF8867801B029A187D
:107B00006A840A7A4B7A8F7AC87A0D7B65701B0279
:107B10009A183B04D21800061018179FF860487B8B
:107B20008A7BCB7B3B77120210186081087C7877C8
:107B3000487C149A9072887CD072C87C159B18740B
:107B4000087D5874487D11909874C87D0A7E120291
:107B500012181A84887DD87418464B7EC375887EA7
:107B6000CD7E2D022818B880087F4D7F2D02281861
:107B7000F880887FB877C87FF8772020085C149D4C
:107B800028732120085C68732A20085C2A314D780C
:107B90002D0228188D782D044019C978090640183F
:107BA00018998864119801E0EB7DA87C7D498B7061
:107BB0000A8080001F38C882C883139800281FD00D
:107BC00022227748825C034622335B781B029A1894
:107BD0000A842422825C034624335B781B029A18B1
:107BE000CA842622825C034626335B781B029A18DD
:107BF0008A832822825C283040780002801888849A
:107C00006948032569A2294602F0B6FD189F387815
:107C100014907B78B8780F90FA78B8791390F87947
:107C20001190387A1090787AB97A08900991009377
:107C30000F9801900292169803901298049013984E
:107C400005901198069010980790FAA2F8482946D6
:107C5000149B02F091FD3D46643580212846F8F7DB
:107C60007CFAB878C11E02290ED3012800D18FE119
:107C7000022800D0ABE11691149078787F2250430F
:107C8000F7494018F74907E01691149078785B227D
:107C90005043F1494018F14941182846F8F744FA91
:107CA0000D9D1898C6870E34324602E0641C0F2AD8
:107CB0000ADA21780029F9D0491C8907C90F9140B7
:107CC0000E43C687521CF1E71699022907D314996F
:107CD000491E012900D97DE14279D24901E042796A
:107CE000CF4989180C78002D00D177E1C1790E9128
:107CF000032900D94AE14279062A00D979E14921CC
:107D0000890041181191E43010900E98401E129095
:107D100019A800190F9000231392149403E01898E7
:107D2000290600D15AE1052A5AD8C0467A44127968
:107D300052009744455C728598ABC046881300009A
:107D4000E20400000C080000060A0000040F000016
:107D50000000104130C1BD41000070400000F04003
:107D60000000D041120C0000140B000012120000A1
:107D7000140E00000E160000130D00001216000075
:107D80000E120000140B0E0A12080000101600005C
:107D90000E0B0000DC930102DE9301020CA801022D
:107DA00018A80102489401020108000043617365AC
:107DB00020706172616D65746572733A200D0A00FE
:107DC0001693DFB2002F04D019A801223946F8F724
:107DD000BDF9002C00D191E019A8C019BB498AE077
:107DE000E8B2022867D00027022867D06BE00E981F
:107DF000022872D1E8B2022800D103461693DFB2FE
:107E0000002F04D019A801223946F8F79FF9002C59
:107E100074D019A8C019ACA16DE0E8B2022800D155
:107E200004231693DFB2002F04D019A8012239468B
:107E3000F8F78CF9002C61D019A8C0199FA15AE05D
:107E4000E8B2022800D106231693DFB2002F04D037
:107E500019A801223946F8F779F9002C4ED019A853
:107E6000C01992A147E0E8B2022800D10C23169372
:107E7000DFB2002F04D019A801223946F8F766F9BD
:107E8000002C3BD019A8C019874934E0E8B2811E04
:107E90004A424A419700022804D119A801223946D2
:107EA000F8F754F9002C16D019A8C0197CA1224665
:107EB000F8F73AF90FE00627022804D119A80122A1
:107EC0003946F8F743F9002C05D019A8C0198049A4
:107ED0002246F8F729F9169710E01693DFB2002F23
:107EE00004D019A801223946F8F730F9002C05D042
:107EF00019A8C01973492246F8F716F93C193F2C06
:107F000005D80F98C0194021091BF8F726F91298D7
:107F10000228189801D2002002E0C078411E884152
:107F200015990870611E2E46E8B202280CD1179AE6
:107F3000517019A9119AB8C9B8C2B8C9B8C2B8C99C
:107F4000B8C2B8C9B8C20DE0179A117019A9109A31
:107F5000B8C9B8C2B8C9B8C2B8C9B8C2B8C9B8C235
:107F6000C10709D180073546149C139A169B00D48B
:107F7000D5E602208543D2E6FE2035460540189816
:107F8000149C139A169B290628D0CCE637A231E020
:107F90001691149078780B994143334808181F388C
:107FA0006F21C9430D9D7A180378D427D3554378A0
:107FB000D827D3558378DC27D355002900D170E624
:107FC000C378E027D3551031001D189FEBE701203F
:107FD000404A10E00024002D00D087E629B0F0BD13
:107FE00080290ED30F20B87210481799888310206B
:107FF00020E525A20120014602F0BEFB189829B019
:10800000F0BD1020402904D3B8720849179B99830A
:1080100010E5B87204481799888314200AE5C04611
:1080200001BB0000FABA0000150F0000140B00009D
:108030000108000025642025642025642025642093
:1080400025642025642025642025642025642025BE
:10805000642025640D0A0000D9D200001DF7FFFF3F
:10806000F1C9000089FBFFFFE1D100007472785F65
:108070006D6F646520706172616D657465722065F5
:1080800072726F720D0A00004E7366642070617226
:10809000616D65746572206572726F720D0A000001
:1080A000FFFFFFFF01FF00002CBE0000FFFFFFFFEE
:1080B000FF0101FFFF01FF01FFFF01FFFFFFFF01C4
:1080C000FFFF01FF30C00000FFFF01FF4CBE0000BA
:1080D000BCBD00008FC90000002800D1014806493E
:1080E0000860704798900102F0B586B0002805D16D
:1080F0000148006802E0C046F09301023121C90046
:10810000049141188A791F231A40CD79ED06AD0DEF
:10811000AA180D7AED066D0C52194D7AED062D0B4D
:1081200052198D7AED06ED095219CD7AED06AD089A
:1081300052194D7CED075219BD4C22600A7B1A4042
:108140004E7BF606B60DB2188E7BF606760C9219AB
:10815000CE7BF606360B92190E79F606F6099219C1
:108160004E79F606B608921962604A6AB14D2A4005
:10817000A2608A6A2A40E2602D22D20087183A7EE5
:108180001A4003937E7EF606B60DB218BE7EF60642
:10819000760C9219FE7EF606360B92193E7FF60695
:1081A000F60992197E7FF606B60892190E7CF6073C
:1081B00092192261BA7F1A400597FE7FF606B60D26
:1081C000B218049BC35CDB065B0CD2184B78DB0651
:1081D0001B0BD2188B78DB06DB09D218CB78DB06B9
:1081E0009B08D2186261CA692A40A2610A6A2A40C1
:1081F000E2618A7C01252A40CB7CDB079B0F9A1821
:108200000B7DDB075B0FD2184B7D9B07DB0ED21873
:108210008B7DDB079B0ED218CB7D1B079B0D9A181D
:108220000B7E1B079B0CD2184B7E5B06DB0A1343AD
:108230008A7E520612091A43CB7E5B075B08134302
:108240002362CA6A62620A6BA2624A6BE2628A6B4A
:1082500022633922D200835C1E462E4066635E4252
:108260005E41B304AE04744F3C68B443E3183B6012
:1082700083185A782A409C782407E40EA2188C8F21
:108280006401A2186D4C1440C98FC905490A091927
:10829000DA78D207120A89181A791207120989188E
:1082A0005A79D207D2088918FB4EB1639968F163F5
:1082B000997904952940DA79D207920F51181A7BDF
:1082C0005207D20E89185A7BD206920D51189A7B0A
:1082D0005207D20C8918DA7BD206920B89181A7CC5
:1082E000D206520A89185A7C520792090A43997C8D
:1082F000C906490851183164D97C039A11401A7D86
:10830000D206920D51185A7DD206520C89189A7DC8
:10831000D206120B8918DA7DD206D2098918716447
:10832000197E0F2421405A7E120151189A7E1203A1
:108330008918DA7E1207120A51181A7F12071209D9
:1083400089185A7F12078918B164997F01942140D6
:10835000DA7F1207120E51183D22D200835C5B07B0
:108360005B0D5918841862781207520C8918A2788C
:10837000D206120B8918E278D206D2098918F16464
:10838000217907220A406179C9008918A279520629
:10839000920B5118E2799207120B8918227AD207B0
:1083A0008A18BF490A60627AA37A1B029A18E37A94
:1083B0001B04D2184A60E289BA4B13400394228A04
:1083C000D2049209D2188A6003463033598CB64AD7
:1083D000114002939A8CD205D20A51185622825C1F
:1083E00012068918B14D2960014656314A788C78B9
:1083F0002402A2188C8864056409A218CC7824078A
:1084000012196A60CA880C7AA407A40BA2184C7AC5
:108410006407E40A1219AA604989E96049218900C0
:108420004118FF226632821800921035002207E0C0
:1084300000300040FFFFFF0004040040FF3F000049
:1084400084186427E65D03273E406523E35C9B07B1
:108450001B0F9B196626A65DB607B60EF318672696
:10846000A65DB601F318DBB26826A65DB607B60DA9
:10847000F3186926A65DB607360DF3186A26A65DC1
:10848000B607B60CF3186B26A65DB607360CF318C4
:108490006C26A65DB607B60BF3186D26A65DB6076B
:1084A000360BF3186E26A65DB607B60AF3186F26CC
:1084B000A65DB607360AF3187026A65DB607B6099C
:1084C000F3187126A65DB6073609F3187226A65D65
:1084D000B607B608F3187326A45DA407E31808C509
:1084E0001032802AACD1019AD243704EB4180B7866
:1084F0003B404D78AD072D0FEB188D78AD07AD0ED5
:10850000EB18CD78AD01EB18DBB20D79AD07AD0DF1
:10851000EB184D79AD072D0DEB188D79AD07AD0C2E
:10852000EB18CD79AD072D0CEB180D7AAD07AD0B1F
:10853000EB184D7AAD072D0BEB188D7AAD07AD0A10
:10854000EB18CD7AAD072D0AEB180D7BAD07AD0901
:10855000EB184D7BAD072D09EB188D7BAD07AD08F2
:10856000EB18CD7BAD07EB18A3641031121DBDD104
:10857000009B19785A785207520D51189A78D207F1
:10858000120D8918B164059B1968F164D97D5A6888
:108590001202511831659968454A0A40998A49057D
:1085A00089187165D9683D4C2140B1651969214030
:1085B000F165029E3178049D294082785207120F9E
:1085C0005118C2799207920E8918427A9207920D39
:1085D0005118827A9207120D8918C27AD207920C2A
:1085E00089189A7DD207520C891872789207D20B9B
:1085F0008918B2781207D20A8918F2781207D209BC
:108600008A182C490A60327C737C1B071B0D9A1850
:10861000B37C9B069B0BD218F37C1B079B0AD218DA
:10862000337DDB065B09D218737DDB071B09D2188B
:108630004A60B27D2A40C38F5B009A188A60826CC0
:10864000CA60C26C22400A61F27D7F231340328CE3
:108650005204520AD2184A6102698A614269CA61A7
:1086600082690A62C2694A62026A8A62426ACA62AC
:10867000826A0A63C26A4A63039A927CD201121D1B
:108680000A64027A3A40CA65808F074A1040086639
:10869000002006B0F0BDC04600300040FFFFFF00E4
:1086A0009C300040FF1F0000FF030000004000401E
:1086B000FFFF1F00002000401A480068806B800800
:1086C0000249096849004018093070471004004009
:1086D0001449096842684A6182688A61C268CA614D
:1086E00003680B6102690A6242694A6282698A62AE
:1086F000C069C8620C4803600C4A13608B699360C0
:108700008360CB69D360C3600B6A136103614B6AFA
:10871000536143618B6A93618361C96AD161C161AD
:108720007047C046F09301020C1000401820004032
:1087300010B52D21C9004118027A032A04D100790D
:10874000002807D0082006E08378DA1E022A05D226
:10875000032412E0142088601C203DE0012B02D18C
:10876000C8228A6012E00479042C01D3462404E074
:10877000032C01D1322400E014248C605B1E022BF8
:1087800004D3022A10D24279154B01E04279154BED
:108790009B181B78402B04D0102B06D114234424A3
:1087A00005E02A233E2402E04279342348244B800A
:1087B0000C80022A06D0062A08D0052A08D11822E1
:1087C0004C2301E0142250230B8000E01C224A803D
:1087D000C078042803D1142048806420088010BD8C
:1087E00001BB0000FABA0000134800687047C04699
:1087F00010B5104A107091700F49002813D05068BE
:108800000861042048619078FF2212020B4B1C681B
:108810009443800380B20019186001204007084A81
:108820001060084A106000200860074901220A60B1
:1088300010BDC046E0930102180400401CE400E0B3
:1088400080E200E000E100E070000040F0B591B08F
:10885000002801D1C04800688778F91E022913D387
:10886000012F21D0022F3CD11021CA434478214648
:10887000193991423DD800970125B94A2846294621
:10888000234601F079FF53E10821CA434478214689
:108890002139914218D800970125B14A2846294626
:1088A000234601F069FF43E10821CA434478214689
:1088B0000939914234D800970125A94A284629460A
:1088C000234601F059FF33E1032F3CD0042F43D15D
:1088D000C3780125042B00D02DE106462A0204238B
:1088E00043E00125A6A2284629463B4601F044FF65
:1088F0001EE1C3780125052B0AD806462A02284620
:1089000098401B21084230D10021052B08462ED06B
:1089100002200090914A2846294601F02DFF07E1E8
:108920000646C3780021022B1ED3032B1CD0042B38
:1089300008460A461BD001250095884A2846294644
:1089400001F01AFFF4E0C3780125032B00D0FAE010
:1089500006462A02032308E0012583A22846294669
:108960003B4601F009FFE3E00A46012148020F916E
:10897000592189007518FD2149007118029131466D
:1089800062313F05D219641E1F2727405C013C1944
:108990001443044332795207D20C22432B789B06AE
:1089A0005B0BD218B379DB071B0B13436D4D2B60A8
:1089B000F279032310931A40737A9B079B0E9A183F
:1089C000B37A5B07DB0D9A18F37ADB079B0DD2189D
:1089D000337BDB075B0DD218737B1B075B0CD21854
:1089E000AA603269EA6072692A61B2696A61F269F1
:1089F000AA61326AEA61726A2A62B26A6A620F988E
:108A00000870F06AA8623F20C4432C353046E43039
:108A10000F903046E5300E903046E6300D903046EF
:108A2000E7300C903046E8300B903046E9300A9041
:108A30003046EA3009903046EB3008903046EC3052
:108A400007903046ED3006903046EE3005903046C7
:108A5000EF3004903046F03003903746F13730461F
:108A6000F230F3360F990A194021525C109B1A40DC
:108A70000E9B1B195B5C9B071B0F9A180D9B1B1908
:108A80005B5C9B079B0E9A180C9B1B195B5C9B0104
:108A90009A18D2B20B9B1B195B5C9B079B0D9A1813
:108AA0000A9B1B195B5C9B071B0D9A18099B1B19E2
:108AB0005B5C9B079B0C9A18089B1B195B5C9B07D4
:108AC0001B0C9A18079B1B195B5C9B079B0B9A1846
:108AD000069B1B195B5C9B071B0B9A18059B1B19BC
:108AE0005B5C9B079B0A9A18049B1B195B5C9B07AA
:108AF0001B0A9A18039B1B195B5C9B079B099A181E
:108B00003B195B5C9B071B099A1803195B5C9B076D
:108B10009B089A183319595C8907891802C51034C3
:108B2000A0D102980078042101430E48C1630025BA
:108B3000284611B0F0BD04200090084A2846294676
:108B400001F01AFEF4E703200090044A2846294663
:108B500001F012FEECE7C046F093010264C9000088
:108B6000AAC9000000100040556E646566696E6514
:108B700064206D65616E205052462025640D0A0008
:108B8000496E76616C6964206D65616E2050524655
:108B90002025640D0A0000007047704780B50E491B
:108BA0000E480246083A1268920000D460314268CA
:108BB0000A4342600A490A6808239A430A60091F67
:108BC000012252040A600321890402688A43026078
:108BD000FBF716FB80BDC046200000802800004047
:108BE00004020040B0B5032000072D490A68824303
:108BF000012568071018086000242046FFF7CDFF04
:108C00002046FFF7C9FFEFF31080284002D1EFF3B1
:108C1000108172B68021C943224A53680B405360C9
:108C200093680B409360D3680B40D36013690B408B
:108C3000136153690B405361002800D162B6B0BD87
:108C400070B50C4603210907154A13680B431360DE
:108C50000122EFF31081114002D1EFF3108272B6BE
:108C60008025EA430F4B5E6816405E609E682E4387
:108C70009E60DD681540DD601D6915401D615D6900
:108C800015405D61002900D162B6002802D00120A4
:108C9000FFF783FF002C02D00120FFF77DFF70BD9E
:108CA00000040040489501020D4A002907D001291F
:108CB0000BD10121814010688843106007E0012139
:108CC000814010680843106001E001218140101FBD
:108CD00002680A430121C907114301607047C04679
:108CE00044000040032804D840000649085A00B256
:108CF0007047002000B27047032802D84000014AA4
:108D00001152704746A80102B34908707047C04627
:108D10001348203080210122026042608260C260DC
:108D2000026142618261C261031F1A600346083B0F
:108D30001A6003460C3B1A600346103B1A60034658
:108D4000143B1A600346183B1A6003461C3B1A602A
:108D50000346203B1A60103940300029DBD17047B0
:108D6000F0A0010270B58AB00C460546FF20FC3029
:108D7000A8490E68315C59208000335CB2783078A5
:108D800008AE069609AE05960C4E04962126760688
:108D900003960B4E0296012601960E2600965B1C4A
:108DA000DBB2F9F7F7FA0998F7F70CFD2870089885
:108DB000F7F708FD20700AB070BDC04600002041E2
:108DC00000000443F0B58BB00446457C824800782F
:108DD0008249002822D000200880814A1080814BDF
:108DE00001269E761E830A907F4800787F4E367853
:108DF0006DB205957E4D04957E4D03950AAD0295A5
:108E00007D4D01950096F9F703F80A9D1120205633
:108E10007A497B4A00F0BAFB064626E000260E801F
:108E20006F4A16806F4B01209876188309966E481A
:108E300000786E4F3F786DB205956D4D04956D4D80
:108E4000039509AD02956C4D01950097F8F7E0FF89
:108E5000099D112021567F20C005009001900296A7
:108E6000664A674B3046FAF727F943200106284641
:108E7000F7F7DEF9F7F7A6FC0890624800780028BB
:108E800024D05120800060494A7D42438D185F48BC
:108E90000068A8642F46403750480078B87450489E
:108EA0000078F8745548007838755548007878751A
:108EB00057480078F87550480069F7F783FCB87593
:108EC00052484069E8644C4800686864FF20FE30FE
:108ED00050490968085C3922D2008918022812D347
:108EE00003D04E48007801280DD14B480660434816
:108EF00000883A4A108042480088394A1080092088
:108F00000790089605E04448089A02603548C08BEF
:108F100007900B780022002B01D0114600E0D143CE
:108F20000125002B01D0042300E0EB43A67AAD1B02
:108F3000EE175B1971416568AE0F277AAD00ED1928
:108F40005641677A3F1FF817ED1970414000EE0F48
:108F500080196D00EB1848418001990E4118980165
:108F600027239B02C31A91411D4805881B4800888E
:108F7000854201D00798421B10202056C001194D90
:108F80002D8C032D07D1E468E5176D0A6419E415EB
:108F90000519EC170FE0E468E5176D0A6519EC1781
:108FA000ED15C6174519744197B2002F00D034460D
:108FB000002F00D00546581BA141130409D012B25E
:108FC000D2015242D31780185941089BDA17C01AB0
:108FD00091410BB0F0BDC04686930102FCA6010290
:108FE000FAA60102489401029590010294900102B0
:108FF000E89C0102E89A010200A701024AA70102C7
:1090000048A70102B4A00102EC9D010264200040C7
:10901000F8A60102F0930102F4A601024CA7010296
:10902000C10D4002803070470120C0071B49086015
:109030007047C04610B519480068C10710D18107B4
:1090400011D4410712D4010713D4C10614D48106E8
:1090500015D4410616D48021084016D031A215E05F
:1090600001240FA213E0022411A210E0032414A291
:109070000DE0042416A20AE0052419A207E0062444
:109080001CA204E0072421A201E0254A04090220D1
:10909000032101F071FB204610BDC0465C0000407A
:1090A000526573657420627920504F520D0A00009A
:1090B000526573657420627920424F520D0A000098
:1090C00052657365742062792050494E0D0A000084
:1090D0005265736574206279205744540D0A00006C
:1090E0005265736574206279204C4F434B55500D87
:1090F0000A0000005265736574206279205357207E
:109100005265626F6F740D0A00000000526573654E
:1091100074206279205359535245510D0A000000C2
:109120000EC600005265736574206279204456446F
:10913000440D0A0001218140044A1F2802D0106812
:109140008843106010680843106070471C0000409E
:10915000F0B583B0029104469949F6F7BBFF054686
:10916000984901942046F6F7B5FF97494618974964
:10917000714300956F189649441864212046F6F70C
:10918000A9FF3818A108471A92492046F6F7B8FFF8
:10919000381891494518914F05D464213046F6F7A7
:1091A00099FF0C4614E0A6B264213046F6F792FF10
:1091B000B7204000A20701D1002907D1884B734393
:1091C0000422D341874A934200D3401E0C464519DE
:1091D0000098474302980680192001013046F6F7AF
:1091E00079FF2A461F3A284600DB1046019BFF18EC
:1091F000B30705D1002C03D01F2D05DA0120C5E0EF
:109200001F2D0BDA0120C1E005461D3D034600DBA2
:109210002B461C2808DC02201546B7E000290CD09C
:109220001C21451A0CD50CE019461F39184600DBE5
:1092300008461F2B1DDA0320A8E01D21451A00D483
:109240002846002D08D401461F39024600DB0A4695
:109250001F2804DA032099E00220154696E01546FF
:109260001E3D104600DB28461E2A0CDA04200D465F
:109270008CE005461E3D024600DB2A461E280BDA1E
:1092800004200D4682E001461F39024600DB0A46F3
:109290001F280ADA052079E011461F39104600DB45
:1092A00008461F2A0BDA052070E015461E3D1046C1
:1092B00000DB28461E2A0CDA06200D4666E005462D
:1092C0001E3D024600DB2A461E280BDA06200D460C
:1092D0005CE001461F39024600DB0A461F280ADA15
:1092E000072053E011461F39104600DB08461F2AAD
:1092F0000BDA07204AE015461F3D134600DB2B46DC
:109300001F2A0CDA08200D4640E005461F3D0246A4
:1093100000DB2A461F280BDA08200D4636E01946E6
:109320001E39184600DB08461E2B0ADA09202DE0FC
:1093300011461E39104600DB08461E2A0BDA0920AA
:1093400024E01F28054601DB05461F3D1F280CDAD7
:109350000A200D461AE01F28054601DB05461F3D81
:109360001F2806DA0A200D4610E01E2D05DB0C2012
:1093700004E01E2D06DB0C2005E00B201E2D05DB76
:109380001E3D03E00B201E2D00DB1E3D029EB07033
:10939000681CF070E12001013846F6F79BFE307141
:1093A000C0B211494143CC193C212046F6F792FE48
:1093B00070713B21C94341430819B07103B0F0BD3E
:1093C000805101008033E101B207000093FEFFFFEE
:1093D000B107000070FEFFFFA7FA0A0080AEFEFF93
:1093E000295C8FC20BD7A300F0F1FFFFF0B581B06D
:1093F0000446FFF7F7FBA08A1B4FB882B98A002901
:1094000009D0F8820220B87100207882FFF7ECF9C9
:10941000F86101B0F0BDE08A7882A1697A8A1348C8
:10942000F6F782FE2046FFF7CDFC06460D461048B3
:10943000007CFFF757FC81B2C90B401800B2C1177E
:109440004010301A38678D417D67FFF7CDF9B8615C
:10945000607CF871F86D401CF865FEF737F93865E7
:109460000120B87101B0F0BDB096010250A8010210
:1094700018900102F0B581B0EFF3108072B60020B1
:109480000146FBF79DFF0446002803D062B6204644
:1094900001B0F0BD01273A030025074E28463146AA
:1094A000FBF7E8FEBB02054A28463146FCF7C0FB45
:1094B00062B6204601B0F0BD00E00204F2A2010253
:1094C00007480178491C0170C9B2782903D10121EC
:1094D0004170002101700348012141707047C0466E
:1094E000289701021490010270B514460D460646F5
:1094F0001120FBF703F82248042101600C480460A6
:109500001E4805608660002E0DD0FF200006094928
:109510000A6882430120C007101808600648082125
:109520000160064801601A200221FFF7BDFB70BDF3
:10953000ECA8010200E400E080E200E000E100E0CD
:109540000C4908607047C04610B5044609480068D9
:1095500060430949F6F7D4FD0019084948600848F6
:109560000022026002460C3A4B68136009680160F1
:1095700010BDC046E8A8010240420F000890010259
:109580002C10014000480047C100000080B582B0A7
:1095900013460A4600900348011D0348F9F738FDB9
:1095A00002B080BD28A90102209A010210B50C4921
:1095B0008A1C90420DD2401E0D4A50600D4803682F
:1095C0000B4003218C071B19036000209060116081
:1095D00010BD04480449E622044B00F06FF8C04671
:1095E000FFFFFF00E5C50000FFC50000CBC5000080
:1095F00010E000E020ED00E0B0B50120EFF31081B5
:10960000014002D1EFF3108272B6124A1368124C75
:10961000226864688506114800682840850E5D1937
:109620002923DB006B43002C1D4606D1002809D1FD
:109630001E20684300290AD0B0BD121BD218551C49
:109640000028F5D01D461E2068430029F4D162B6DB
:10965000B0BDC04658B4010214E000E004ED00E0E3
:1096600080B50020FBF756F9404280BDB0B586B00A
:10967000104869460A4638C838C238C838C200247B
:109680002046FBF74DF903992046FBF7E3F90198D3
:10969000012803D00824002804D102E00424002873
:1096A00000D104460220FAF731FFE0400249086089
:1096B00006B0B0BD08BB00006CB4010290B01C46FF
:1096C00005AB07C3EFF31080C00702D1EFF31080A2
:1096D00072B6EFF310800B9068460E9070460890BB
:1096E00010AB0F93CF4F3E1D01200490C5023046B2
:1096F0002946224600F0B8FC00213154EFF30380E4
:109700000990EFF308800C90EFF309800D90EFF3D0
:1097100014800A9000F02CFC3868012833D8002807
:10972000C14F00D0C14F2A20C1497A69920703D5A1
:109730000A783A60401E491C0028F6D1B948041D39
:109740002046F6F715FD002807D079698907FAD574
:1097500021783960401E641CF5E70220B5497A691A
:10976000920703D50A783A60401E491C0028F6D1BA
:109770002A20AF497A69920703D50A783A60401ED9
:10978000491C0028F6D1FFF737FF0346AA4A3046A6
:109790002946FDF7D9FE04463018291B089F3B1FB8
:1097A000049A9343A5A2FDF7CFFE9E4909680129BB
:1097B00066D8001900299C4C00D09C4C00280AD087
:1097C0009849091D6269920703D50A782260401EF4
:1097D000491C0028F6D10A209F496269920703D5E7
:1097E0000A782260401E491C0028F6D10598F6F739
:1097F000BFFC002809D061698907FAD5059A11785C
:109800002160401E521C0592F3E7022089496269DB
:10981000920703D50A782260401E491C0028F6D121
:109820000A208EA16269920703D50A782260401E41
:10983000491C0028F6D10698F6F79AFC002809D0B2
:1098400061698907FAD5069A11782160401E521C79
:109850000692F3E7022077496269920703D50A78F6
:109860002260401E491C0028F6D10A207EA16269B0
:10987000920703D50A782260401E491C0028F6D1C1
:109880007CA230462946079BFDF75EFE65490968C4
:1098900001290E9B1BD80029634900D06349002889
:1098A0000AD0604A121D4C69A40703D514780C60D5
:1098B000401E521C0028F6D102205E4A4C69A407C3
:1098C00003D514780C60401E521C0028F6D16AA201
:1098D00030462946FDF738FE04463018291B694AF0
:1098E0003B46FDF731FE4F490968012911D800199F
:1098F00000294D4900D04D4900280AD0494A121D7F
:109900004B699B0703D513780B60401E521C00283F
:10991000F6D15D4A30462946099F3B46FDF714FEC5
:109920000446F800C00FB900C90F7A00D20F0092A8
:10993000019102903019291BFB0F544AFDF704FED8
:1099400004193019291B3F233B40514AFDF7FCFD08
:1099500034490968012911D820180029324900D05A
:10996000324900280AD02F4A121D4B699B0703D5A4
:1099700013780B60401E521C0028F6D1454A304631
:1099800029460B9BFDF7E0FD04463018291B424A8F
:109990000A9BFDF7D9FD23490968012911D800194F
:1099A0000029214900D0214900280AD01D4A121D52
:1099B0004B699B0703D513780B60401E521C00288F
:1099C000F6D1364A304629460C9BFDF7BDFD0446CC
:1099D0003018291B324A0D9BFDF7B6FD1149096865
:1099E0000129114A0DD80019002908D00F4A06E0B4
:1099F0005169890703D531781160401E761C002813
:109A0000F6D128490E98091AA94200D32946890897
:109A100000F03CFE24480068002800D0804700F099
:109A200045F8C04640B501020090014000A0014049
:109A30003FC60000CEC9000028C600000D0A23233F
:109A4000232041535345525420402030782530384C
:109A500058202323230D0A0002C7000046554E4319
:109A600054494F4E3A2000004C494E4520202020BA
:109A70003A200000256400000D0A53503D2530387F
:109A8000580D0A00C7C60000DDC60000E9C6000088
:109A9000D1C6000086C6000095C60000A4C600001E
:109AA000AFC6000000F802023CB50102F7480068AA
:109AB000012811D8002801D00B4800E0FC480C21F7
:109AC0000A4A01E0002907D043699B07FAD51378B9
:109AD0000360491E521CF5E71E20FFF72BFB00BF59
:109AE00000BF00BF00BFFAE700A0014032C600007F
:109AF0008AB00646E448B06600F03AFAFFF77CFD0B
:109B00000346E248041D01200590C502E04A2046B4
:109B10002946FDF719FD074608942018DB4C0995E6
:109B2000E91BF36C3F2206921340DAA2FDF70CFD0D
:109B30002168012910D8C0190029DD4900D0DD496C
:109B4000002809D0221D4B699B0703D513780B60B1
:109B5000401E521C0028F6D1F36BD7A2089C204669
:109B6000099D2946FDF7F0FC0746291A2018336C99
:109B7000069A134007D1D8A2FDF7E6FCC34C216832
:109B8000012907D917E0CEA2FDF7DEFCBF4C216802
:109B9000012910D8C0190029C54900D0C54900289D
:109BA00009D0221D4B699B0703D513780B60401E1B
:109BB000521C0028F6D10027CBA5B80030580090E1
:109BC000089809992A463B46FDF7BEFC2168012901
:109BD0000FD80029B64900D0B649002809D0221D67
:109BE0004B699B0703D513780B60401E521C00285D
:109BF000F6D17F1C0D2FE0D1736BBFA2089C2046CD
:109C0000099D2946FDF7A0FC074620189F4CE91B3B
:109C1000B36BBC4AFDF798FC2168012910D8C01924
:109C20000029A34900D0A349002809D0221D4B696F
:109C30009B0703D513780B60401E521C0028F6D1F9
:109C4000336CB14A089C2046099D2946FDF77CFCEF
:109C50000746326CD000C00F9100C90F5300DB0FD4
:109C6000009301910290E019E91BD30FA74AFDF779
:109C70006BFC3246C619A019A91B1546136C069A2F
:109C80001340A34AFDF760FC80490968012911D8F7
:109C900080190029864900D0864900280AD07B4ACD
:109CA000121D4B699B0703D513780B60401E521C95
:109CB0000028F6D12E466B6C964A089C2046099DDA
:109CC0002946FDF741FC07462018E91B0796B36CAF
:109CD000914AFDF739FC6D4A1168012910D8C01965
:109CE0000029734900D07349002809D0121D4B691F
:109CF0009B0703D513780B60401E521C0028F6D139
:109D00000798426E042360215C2004931A400B469E
:109D100000D003460693002A00D00846079E335819
:109D20007E4A089C2046099D2946FDF70DFC074602
:109D300006983358E019E91B794AFDF705FCC61966
:109D4000A019A91B079A536E76A2FDF7FDFB4F4998
:109D50000968022911D280190029554900D05549B6
:109D600000280AD0494A121D4B699B0703D5137876
:109D70000B60401E521C0028F6D10798C36C0646A3
:109D80006DA2089C2046099D2946FDF7DDFB07468C
:109D90002018E91B336D6B4AFDF7D6FBC619A019D5
:109DA000A91B079F7B6D68A2FDF7CEFB8619A01942
:109DB000A91BBB6D67A2FDF7C7FB344909680129E0
:109DC000059C11D880190029394900D0394900284B
:109DD0000AD02E4A121D4B699B0703D513780B60DE
:109DE000401E521C0028F6D10798476B5D4A9742E7
:109DF00037D2032087430026059CB000395802461D
:109E0000049B1A43BA5808230343FB580C25054307
:109E10007D5900910192029303953B180898099986
:109E2000514AFDF791FB1949096801290FD800290A
:109E30001F4900D01F49002809D0089A4B699B0789
:109E400003D513780B60401E521C0028F6D11B2E40
:109E5000444A06D80798406B361DB100401890421E
:109E6000CBD30798406B111A099A914201D88908FF
:109E700000E0610200F00AFC3C480068002800D0C5
:109E80008047FFF713FEC04622224B4D40B501022A
:109E900028C600000D0A0D0A2323232045584345F8
:109EA0005054494F4E202564202323230D0A0000DF
:109EB0000090014000A0014050433D25303858003B
:109EC0002C20457863657074696F6E4E756D6265A0
:109ED000723D25640D0A00002C205468726561648F
:109EE0004D6F64650D0A000052252D32643D25300A
:109EF00038580D0A0000000053503D253038580DE9
:109F00000A000000C7C60000DDC60000E9C6000068
:109F1000D1C6000086C6000095C60000A4C6000099
:109F2000AFC600004558435F52455455524E3D253B
:109F30003038580D0A000000494353523D2530384F
:109F4000580D0A00BAC600005343523D2530385818
:109F50000D0A00004343523D253038580D0A0D0AC2
:109F60000000000000F802026AC600003CB50102D1
:109F7000F0B583B0344D2C68012C06D8601E8441A6
:109F8000204601F0ABFA0028FAD10120EFF310814E
:109F90000140019102D1EFF3108072B62B48285A8C
:109FA0002B49695A814245D02A68002A01D02A4E9D
:109FB00000E0284E1F23DB020293284C022A27D2FE
:109FC00005E01046214AA85282B2914232D087B2AF
:109FD000B9420A4600D8621C131A21482B521804B1
:109FE0000DD0E819001D9FB201E0002F07D0736962
:109FF0009B07FAD5037833607F1E401CF5E7A24229
:10A00000DFD902981018DDE7304683B299420CD0B0
:10A01000024680B281420E4600D8661CA642F3D9A1
:10A020000298301883B29942F2D108496852B01AA6
:10A030000B4968520B48002129540198002800D18F
:10A0400062B603B0F0BDC04640B501020A08000088
:10A05000080800000090014000A00140FF07000038
:10A060000C0800000F080000F0B58DB007931746EC
:10A0700000240C9409AA13C215E006986849F6F763
:10A08000D7F8F6F79FFBC117401848406549F6F727
:10A0900021F8009509A806223346F9F74FFEBDE0E6
:10A0A000002C00D5BEE138787F1C25280DD0002873
:10A0B00000D1B7E10B9A511C0A9B9942F0D8099B39
:10A0C0009854641C0C940B91EAE7089400253978A5
:10A0D00023390D2914D801207944097949008F4486
:10A0E000090F0F0F0F0F0F0F0B0F060F0F0D05436B
:10A0F0007F1CECE70820FAE70420F8E70220F6E7E7
:10A100003878014630390024092902D926463946D3
:10A110000BE000260A2171430E18303E791C787836
:10A120000246303A0A2A0F46F4D32E2817D14A1C89
:10A13000487801463039092905D911464F1C253880
:10A14000532811D96AE000240A2161430C18303CDD
:10A15000511C50780246303A0A2A0A46F4D34F1C62
:10A160002538532800D959E04000C04678448088FB
:10A1700040008744A0005300530053005300530095
:10A180005300530053005300530053005300530037
:10A190005300530053005300530053005300530027
:10A1A0005300530053005300530053005300530017
:10A1B00053005300530060005300530053005300FA
:10A1C00053005300530053005300530053005300F7
:10A1D00053005300530053005300980053005300A2
:10A1E00053005300530053005300530053005300D7
:10A1F000AD00B600530060005300590053005300F7
:10A2000053005900530053005300DE005300530025
:10A21000BD005300D3005300530098000C9C3FE74F
:10A220000024744940420F00791C38780F462538C5
:10A230005328F3D898E70799C91D07208143086878
:10A2400007914968F6F74CFB00210690F6F71AFAD9
:10A2500000280BD10B99481C0A9A904206D8099AFB
:10A260002D2353540899491C0C910B9007980830E2
:10A2700007900698F6F7A6FA0095C2178118514084
:10A2800009A822463346F9F759FD0B98411C0A9A52
:10A29000914200D9F1E6099A2E2313540B910C98A0
:10A2A000401C0C90E9E6079802C8079000960195BB
:10A2B00009A8102239E00B98411C0A9A9142ADD8A6
:10A2C000099A252313540B910C98401C0C90A5E778
:10A2D0000B9A511C079C201D0A9B994239D9079063
:10A2E0009CE7079802C80790009509A82246D3E684
:10A2F000079901C9079109990A9A089E02E0401C32
:10A30000002E8BD40378002B88D00B9D6C1C9442BC
:10A31000F5D84B55761C0C960B94F0E7079802C8BD
:10A3200007900096019509A80A222346F9F7A4FD93
:10A3300074E7079B10CB102C079308D3002021460D
:10A34000401C0A09FF291146FAD806280AD8082015
:10A3500009E02368099CA354089A521C0C920B91A3
:10A3600007905BE7401C069009230C980B9D099908
:10A3700005910A9E04940DE0202104463046059E76
:10A38000715506462046049C401C1546014608911E
:10A3900000290AD45B1E0699994206D26A1CB24271
:10A3A000EAD9089908910029F4D50C900B950898E2
:10A3B000002800D532E70126082501E06D1E360190
:10A3C000022DFBD220463146F5F784FE0F28F6D841
:10A3D0000C980590099803900A9806900B9D2046CA
:10A3E0003146F5F777FE691C069A914204D908991F
:10A3F000089100290CD511E00C4A125C039B5A55B8
:10A40000089A521C0D46059211460891002905D460
:10A410007043241A3009102E0646E0D205980C909D
:10A420000B95FBE620460DB0F0BDC0468CBD00008C
:10A4300070B588B00022032803D9D243104608B073
:10A4400070BD804CC44D2A510F4B104EEE508123ED
:10A450001E010123AB5528602C1962600128EDD83C
:10A46000079300220692059204920323039302921B
:10A4700001920091411E8841694600F0CFFC0246DE
:10A48000104608B070BDC04604080000FFC0FFC001
:10A49000F0B583B00C460023D943012C56DB0746A8
:10A4A00002910126EFF31085354002D1EFF31080C1
:10A4B00072B65849584A505C002800D0A3E0565460
:10A4C0005F48115A5F48105A0196F202161A8142EB
:10A4D00040D832465218A24240DB00930295A64271
:10A4E000354600DB25464C490818001D39462A46EA
:10A4F000F5F71AFEA642484E04DA7919621B301DA0
:10A50000F5F712FE4F48305A001981B24E4A914277
:10A5100001D94E494018029D009B4A49705230466D
:10A520004B4E805D002865D1EFF310850198054002
:10A5300002D1EFF3108072B6374A4148115A4148B0
:10A54000105A884232D1434813524FE00C462046FD
:10A5500003B0F0BD42425218A242BEDA3C4A2E4E2F
:10A56000B25C002A0CD03B4AB25A51188AB2364C1F
:10A57000A242284C029F01D9344A8918314A02E08C
:10A58000244C304A029F3355B152421A89B2884254
:10A5900002D22D488018421C93B23048012130A2CB
:10A5A00000F0EAF83C46002DD1D128E0019F9755F4
:10A5B000884201D82448401C421A90B2800A01D037
:10A5C000019882022348144F3A52386801280DD866
:10A5D000431E9841104B5918091D92B21E4B00F0B2
:10A5E00017FE009B002801D00B488355002D029DCB
:10A5F00000D162B6074808490B54002DA7D162B6B6
:10A60000204603B0F0BD054805A1094A09A3FFF79C
:10A6100055F8C0460E08000040B501027EC7000094
:10A6200074726163655F6F7574707574000000000B
:10A630000E02000054524143452042555359000038
:10A640000A08000008080000FF07000000F8FFFFEC
:10A650000F0800000C080000A5A8000002FF000081
:10A660000D0A5472616365206275666665722069C1
:10A67000732066756C6C2C206469736361726473FB
:10A680002025752062797465730D0A00F0B587B0D6
:10A6900005460026069605960496039602968007C0
:10A6A00001D007B0F0BD019102A8142126A2FCF749
:10A6B0004BFF29490968012911D80029274900D0F1
:10A6C000274900280BD002AA01E0002807D04B69D7
:10A6D0009B07FAD513780B60401E521CF5E70199D1
:10A6E0000029DED0204C3746B8002B58D80724D09C
:10A6F000581EA04204D31B4818181C4A90421CD86C
:10A7000002A814211AA2FCF71FFF134909680129A6
:10A7100011D80029114900D0114900280BD002AAF4
:10A7200001E0002807D04B699B07FAD513780B602E
:10A73000401E521CF5E7761C01997F1C8F42B0D257
:10A74000322ED1D3ADE7C0460D0A4261636B7472FD
:10A750006163653A200D0A0040B501020090014096
:10A7600000A00140FFFFFFFCFFFF0200FEFF010011
:10A77000253038580D0A000081B0F0B5C4B00E463F
:10A7800007464993812000012F49085C002845D0E5
:10A7900002920120050204A82946F5F7DEFCFCB26E
:10A7A0000021C8430C2C3AD8721E032A37D82748F8
:10A7B000005DB042084632D3F80535D50021B80512
:10A7C0000DD404A801904018691AA20022A39B5836
:10A7D0002E4AFCF7B9FE0198F5F7CAFC0146780548
:10A7E0000ED404AF7818691AB20029A3D218121F28
:10A7F0001368264AFCF7A8FE3846F5F7B9FC01466F
:10A80000029A04AE70180C46691A49AB0393FFF71D
:10A810002BFC01193046FFF73BFE00E0002044B05E
:10A82000F0BC02BC01B00847FEF7E6FE034604A8F0
:10A83000019007A22946FCF787FE0198F5F798FCDE
:10A840000146B805BDD5CAE740B50102B1D5000043
:10A8500025313075207C200022C7000078C7000019
:10A8600072C7000051C700001CC700003DC70000B0
:10A870006BC7000064C700005FC7000015C7000079
:10A8800028C7000038C700000DC7000099C70000A6
:10A8900057C7000043C700004AC700002EC700008A
:10A8A00000000000F0B581B00B460120EFF31084EA
:10A8B000044002D1EFF3108172B6990F07D0022045
:10A8C00001212DA2FFF758FF002C3DD141E0224984
:10A8D000224D00276F54224AAB5A224AAE5AF3182F
:10A8E0009EB2F60A01D0204E9B19AB52EFF31086B0
:10A8F000064002D1EFF3108372B6AA5A1C4BEB5AF2
:10A90000934202D116482F521AE06854934201D85C
:10A91000164B5B1C9B1A99B2890A00D0830210481F
:10A920002B52286801280BD8411E8841A918091DFF
:10A930009AB2104B00F06CFC002801D006482F544E
:10A94000002E03D0002C04D001B0F0BD62B6002C64
:10A95000FAD162B601B0F0BD0F08000040B50102A7
:10A960000C0800000A08000000F8FFFFFF070000C5
:10A9700008080000A5A800005541525420457272F5
:10A980006F722025780D0A0010B50446FEF72AF9EB
:10A99000A08A002800D010BD0A4CA06D401CA06504
:10A9A000FDF722FF6062606D002805D0FDF71CFFF7
:10A9B00060660020606510BDA069206601206065AA
:10A9C00010BDC046B096010270B5012801D9012022
:10A9D00070BD48224243734B9C58A5691F218D438B
:10A9E000A5610625A5600F2525629C18A27C002A7A
:10A9F00005D1627C002A02D1227C002A14D063682F
:10AA0000002B11D4251D0B40012216469E400C4BF5
:10AA10001E60BFF34F8FBFF36F8F2B68002B03D4E3
:10AA20000B409A4007490A60002803D0012804D14E
:10AA3000092000E00820F9F759FD0020A06170BD51
:10AA400080E100E080E200E0F0B585B00D460278DC
:10AA5000E348C368934219D0446D944216D083688A
:10AA6000934203D0016D914200D07FE09B1A591EA2
:10AA70008B41049348215943032D46D14418E16981
:10AA800000294ED01C34002020606DE09B1A5A1E15
:10AA900093410493032D1AD1039548225A438418F5
:10AAA000A26B0121EFF310850D4002D1EFF3108767
:10AAB00072B6A7691026B743A761A669002E01D117
:10AAC00018342160002D00D162B6039D0CE04821AE
:10AAD0005943421891691832302902D0116810295F
:10AAE0004CD1802111600022482159434018002197
:10AAF000816301628162243000210160002A33D029
:10AB000004A82946904705B0F0BD42189169183253
:10AB1000302902D01168202939D18021116000220A
:10AB200016E00395E26B0126EFF31085354002D164
:10AB3000EFF3108172B6A1692027B943A161A16921
:10AB4000002901D118342660002D00D162B6039D82
:10AB50004821594340180021C163C162416330302C
:10AB600000210160002ACBD105B0F0BD00920E4A51
:10AB70002E329C480D490E4BFEF7A0FD1068009345
:10AB8000019098480949084A0A4BFEF797FD10685A
:10AB900000930190044A243292480449054BFEF781
:10ABA0008DFDC04688940102B1020000FDC700007F
:10ABB000D2C70000B6C70000F0B585B004904821A8
:10ABC0000A464243864B9C58E6690F2535409A1841
:10ABD000167C002E31D04F2040026169014200D125
:10ABE00085E0A06904218843A06102202062012041
:10ABF00081076918D161D36BEFF31084044002D14F
:10AC0000EFF3108572B695692026B5439561956975
:10AC1000002D00D173E010463C30002C00D162B60C
:10AC200000240460D4625463303200201060002B92
:10AC300063D004A8984705B0F0BD0C2D5DD8C04680
:10AC40007D442D796D00AF4467586B580658A16359
:10AC50005858585806009569202D04D015461835C7
:10AC60002D68302D49D1156B566B3432AE4217D258
:10AC70006669360714D5646815686E1C166048430B
:10AC80001818C06A445504980C4644431A19156BA9
:10AC9000566B3432AE4203D21C5966693607EAD489
:10ACA0001268AA4229D14143585882690524A24317
:10ACB00082615A18D36B0121EFF31080084002D152
:10ACC000EFF3108472B694692025AC4394619469C3
:10ACD000002C02D114461834216014463C3400285C
:10ACE00000D162B600212160D16251639CE70C2D36
:10ACF00000D176E7012D00D173E705B0F0BD154610
:10AD00001835286010463C30002C00D187E787E7D3
:10AD10000420206205B0F0BD0120206205B0F0BD26
:10AD200008252562164618369569102D02D035681B
:10AD3000302D4BD10396566A15462835976AB7428F
:10AD400028D1A06902218843A061936B0121EFF310
:10AD50001080084002D1EFF3108472B6039E34686D
:10AD60001027BC4334603468002C00D13160144695
:10AD70003834002800D162B60021216029601162B8
:10AD8000243200201060002BB7D052E7022020624E
:10AD900005B0F0BD2A68B242AFD262699207ACD565
:10ADA0002A68561C2E6048431818006A805C206090
:10ADB00004980A4642439D18AC6A6E6AB4429CD21B
:10ADC00028359C5862699207EAD496E7316800906A
:10ADD0000191044804A1094A09A3FEF76FFCC0468B
:10ADE000889401029CC70000756172745F6972717A
:10ADF0005F68616E646C6572000000003D030000D6
:10AE00005561727420256420737461746520676FC6
:10AE100065732077726F6E6720256400F0B585B08A
:10AE20000E460546022804D3002E02D1012005B0AB
:10AE3000F0BD002D03D0012D08D1092400E0082425
:10AE40002046F9F75BFB2046FEF774F94821694379
:10AE5000E74A505883691F240294A3438361062361
:10AE600083600F230193036257180023BB62BB6307
:10AE7000FB633B627B62FB623B63317F3974727FB1
:10AE80007A74B27FBA7404937B637368B268F468AF
:10AE9000920022435B1E032B0ED8C0467B441B79D5
:10AEA0005B009F4401050307082304E0282302E018
:10AEB000182300E038231A43C260C907090F7269DA
:10AEC0009201D2B28918B2699207920E8918491C70
:10AED000816079613169012901D122210161012D4E
:10AEE0005CD831680E2959D23846123003900324B9
:10AEF000002D01D0204600E004204C432D490E19BE
:10AF0000B178F9F78BFB3968CA6880251046284369
:10AF1000C8602848005D73781B021818C862AA43ED
:10AF2000CA60F9F7C3FB03980078002809D13846B6
:10AF300011300078002804D13846103000780028FD
:10AF400027D07868002815D4032102468A431B497C
:10AF500053588407E40EFF26A640B343A5401D4383
:10AF600055500299014001208840A24908601449C7
:10AF700008600EE08107C90EFF228A40019C044050
:10AF8000083C032084430C48235893438D401D43C1
:10AF900025500120B861049805B0F0BD024803496E
:10AFA000DA22034BFEF78AFB9CC700000FC80000A3
:10AFB000ECC7000020BB00001CED00E000E400E056
:10AFC00000E100E0F0B58FB00E900125002900D11E
:10AFD0004BE0039304910592002A00D145E0012142
:10AFE000EFF3108201910A4002D1EFF3108172B6A3
:10AFF0004827029747437E49CE19B5690023302D73
:10B0000023D831461831C0467D442D796D00AF44B8
:10B0100020242626262626262626262626262626D8
:10B020005E26262626262626262626262626262688
:10B0300018262626262626262626262626262626BE
:10B0400018000223002A0CD00CE0402D01D0802DE6
:10B0500005D10123002A04D004E020240C60002A3A
:10B0600000D162B61D46002B02D028460FB0F0BDBD
:10B07000002575630399F1630499F16205993163C1
:10B080005B4CE35959691322D202114205D00621C3
:10B0900099600F21196271699960317C00290CD087
:10B0A000F56109950895079506950D950B95022173
:10B0B0000A91012810D017200FE0717C9A690029AD
:10B0C0002CD0952002439A6128460FB0F0BD302461
:10B0D0000C60002AC5D0C5E71920049F0C90706849
:10B0E000002805D41F210840019981404148016092
:10B0F00014209861B06806A9F9F748FB0E980299E8
:10B100004143601880686158F34A0092091D3A462D
:10B11000059BF9F7ABFB28460FB0F0BD343611069E
:10B1200002D580218A439A6131680025059A9142AF
:10B130002DD205955D694F214A0215421BD1E905C3
:10B1400002D4029CEC4F0AE0596833685C1C3460FE
:10B15000029C6043E84F3818C06AC1540E982146DB
:10B1600041437E18736B346BA34238D234367B581C
:10B170005D691542E3D002211962019EB10729439E
:10B180003546DD4CEFF31082324006D008E0294608
:10B19000019EEFF31082324002D1EFF3108372B6BA
:10B1A000029B4343E01883692024A343836183699E
:10B1B000002B05D0002A08D0C26B002A0AD154E720
:10B1C000034618331E60002AF6D162B6C26B002A0D
:10B1D00000D14AE70EA8904728460FB0F0BD294697
:10B1E000059D019E3C46EFF310823240D5D0D7E753
:10B1F0008894010280E200E080B5012002496422C7
:10B20000024BFFF7DFFE80BDE4950102F9B10000BB
:10B21000F0B591B010900126002900D19BE0039376
:10B220000591002A00D196E007900121EFF31080EC
:10B230000291084002D1EFF3108172B604924823C4
:10B24000069307994B43AC49C9188D690026302DE8
:10B250006ED80C461834AD00374602A675593E46E6
:10B26000AF46C04639B3000041B3000045B300000B
:10B2700045B3000045B3000045B3000045B30000EE
:10B2800045B3000045B3000045B3000045B30000DE
:10B2900045B3000045B3000045B3000045B30000CE
:10B2A00045B3000029B3000045B3000045B30000DA
:10B2B00045B3000045B3000045B3000045B30000AE
:10B2C00045B3000045B3000045B3000045B300009E
:10B2D00045B3000045B3000045B3000045B300008E
:10B2E00045B30000D7B3000045B3000045B30000EC
:10B2F00045B3000045B3000045B3000045B300006E
:10B3000045B3000045B3000045B3000045B300005D
:10B3100045B3000045B3000045B3000045B300004D
:10B3200045B3000029B30000022600280CD00CE031
:10B33000402D01D0802D05D10126002804D004E045
:10B3400010252560002800D162B6002E069D6A4FA8
:10B35000049C079802D0304611B0F0BD00268E62E2
:10B36000039A8A63059A0A624C620A7C002A0BD00F
:10B370000C960B960A96099608960E9602220D9246
:10B3800001282DD018202CE08A7C2831002A3BD0BF
:10B390000A68A24216D22B464343FA585469A407BE
:10B3A00010D50868441C0C60F918096A085C106024
:10B3B0001098294641437A1811462831936A526AF7
:10B3C0009342E8D345437859816982220A438261D6
:10B3D000304611B0F0BD302525600028B4D0B4E768
:10B3E0001A200F90C86808A9F9F7D0F910984543BA
:10B3F0007A597819C0683849009105992346F9F7B8
:10B4000035FA304611B0F0BDFB589A69140602D5E2
:10B410008024A2439A610A680026049882422ED2B0
:10B420005D694F225202154207980AD00221196223
:10B43000029EB10729431FE028315D6915423E464F
:10B44000F4D137465C69A40702D406992A4E0AE073
:10B450000C68661C0E6006994843274E3018006A37
:10B46000005D186010984143735871188C6A4E6AD9
:10B47000B442E1D329463E46069D1F4F01E03146C6
:10B4800007985A6A002AFCD1EFF31082029B1A40F7
:10B4900002D1EFF3108372B6454378198369102403
:10B4A000A34383618369002B05D0002A09D0826BF6
:10B4B000002A0BD14FE703461833029C1C60002A78
:10B4C000F5D162B6826B002A00D144E710A89047FC
:10B4D000304611B0F0BDC04649AA000048214143A2
:10B4E000054842189269D20601D40020704740589E
:10B4F000416901200840704788940102F0B587B087
:10B5000001460127022505283A4600D02A46002098
:10B510000929014600D01146C900374A54180E21A6
:10B520000591615EFDF7E8FB1026A15F3846FDF747
:10B53000E3FB1227E15F2846FDF7DEFB06951425A5
:10B54000615F03200490FDF7D7FB0598235EA05FA1
:10B55000E15F625F00AD07C528A2069F3846049DE3
:10B560002946FFF709F92046263004263146FCF724
:10B5700055F82620235E2820205E2A21615E2C2299
:10B58000A25E00900191029224A238462946FFF75C
:10B59000F3F827463E3738463146FCF75DF83E2043
:10B5A000235E06983C5EB95F0622BA5E0094019164
:10B5B000029221A207462E462946FFF7DDF85624BF
:10B5C0000D4D285FFCF73CF82B5F2C4621A2384636
:10B5D00031463546FFF7D0F8264658363046FCF758
:10B5E0001BF85820235EF05F00901FA238462946C2
:10B5F000FFF7C2F807B0F0BD889A0102546F4620E9
:10B60000616E742064656C61797320256420256403
:10B610002025642025640D0A0000000050446F417D
:10B620002064656C6179732025642025642025647D
:10B630002025640D0A00000050446F4120676169B5
:10B640006E732025642025642025642025640D0A5E
:10B650000000000050446F4120616E7420737061DF
:10B6600063652025640D0A0050446F4120616E67B8
:10B670006C65206F6666736574732025642025648D
:10B680000D0A0000F0B587B01546774B1A680F24F5
:10B69000A2432F783A431A60744C23462C3B744AD9
:10B6A0001A60049003462246283A12681207FAD517
:10B6B000704E092F0291039306D97249316071606F
:10B6C0000C2F09D171480FE0042F07D96C49316064
:10B6D0006C497160092F06D36D4805E066483060FB
:10B6E0007060664800E068486A490860EB7AFF2BA2
:10B6F00002D10020B0620AE003210B406648C05C22
:10B7000040220243B2620220644AFFF735F8039FE9
:10B710000021384605952A460B46FCF709F80646EF
:10B72000022503215EA2284601913346FFF724F843
:10B7300006963046FCF7D0FC0121049800910840A1
:10B740002CD13D4033D15C4900283AD1002D1ED088
:10B750006048A062E062206360635F4860625F48A7
:10B760000860152085046E1C8E608D606424204660
:10B770000F46F8F79BFF3E603D602046F8F796FFC6
:10B78000281D38605648032156A2FEF7F5FF05989C
:10B79000007BFBF743F9069807B0F0BD2E4605463F
:10B7A0000698FDF753F8284635463D40CBD02E4647
:10B7B00005460698FCF798FC284635463E49002881
:10B7C000C4D03E4808613E4848613E488861152023
:10B7D000C8613D48016840220A430260072108030E
:10B7E000244B5A698243009840031018586105227F
:10B7F000029842432748036898182F4E766B477883
:10B800000F40995C0907490EC919CA032F4B3340F1
:10B810009A18C90151182E4A8918274A5163264996
:10B82000896B3822914382785207920E891804223C
:10B830000A4321498A630F4E31690279019B1A40FC
:10B84000C0784007C00E80181F229143081830614D
:10B8500055204003411C216020606420F8F726FF3A
:10B860001549002D93D073E7040400402C6000407C
:10B8700000040080000600400F040F04A1C1000076
:10B880000304030400040004D2C2000070C00000DE
:10B8900003C40000F493010234C500001DC8000079
:10B8A00050485920706172616D7320736574732004
:10B8B000253038780D0A00009060004012A83E0044
:10B8C0009DD79B5AD579BD49340200403F0080FF87
:10B8D000404000002008820002D50F0002025500FF
:10B8E000020800007577625F72785F696E69740D97
:10B8F0000A000000B0B51820FDF71CFC1920FDF768
:10B9000019FC002420462146F8F75EFB204621461C
:10B91000FBF708F8012503217F2328460A46FBF799
:10B9200019F92846FBF7BEFA0220FBF7E1FE28468C
:10B930002946FCF75DFF2046B0BDF0B581B0164644
:10B9400000910446002001273946FDF779F9EFF30D
:10B9500010853D4002D1EFF3108072B627204001E0
:10B9600070430A21F4F7B6FB0246002C02D00020F7
:10B97000009901E002200021FBF79AFA0446FBF748
:10B9800061FB002D00D162B6204601B0F0BD000081
:10B9900070B504460E4D29680F2001400629FAD0E3
:10B9A00029680140072912D10120EFF310860640D3
:10B9B00002D1EFF3108072B6FCF716FFFA30A860E0
:10B9C000002C01D0FBF7C0F8002E00D162B670BD8C
:10B9D00000040040F0B581B01D460E460446022A20
:10B9E00009D1012738463946FDF72AF90096002289
:10B9F000384629460FE0174601200021FDF720F9BF
:10BA0000012F04D1009600202946024603E000964B
:10BA1000022000210A462346FBF72CFB0446FBF7D5
:10BA200011FB204601B0F0BD70B5002801D0012007
:10BA300070BD0325A9020F4802680F4B5350002424
:10BA40009460012253030D4E3360BFF34F8FBFF359
:10BA50006F8F0B4E336003685A508472048110203C
:10BA6000F8F744FD022007A22946FEF785FE20468E
:10BA700070BDC0461895010251E5CC1A80E100E086
:10BA800080E200E057445420636C6F73650D0A0038
:10BA90002021020C01D010211046020A01D01046CC
:10BAA0000839020901D01046091F820801D010464A
:10BAB000891E420801D0881E7047081A704702E0AC
:10BAC00008C8121F08C1002AFAD170477047002029
:10BAD00001E001C1121F002AFBD17047000084C1A0
:10BAE000000008C10000C03F000038410000AC4128
:10BAF0000000D441280004030000084008000008AA
:10BB000010080408102000000000000000000000E1
:10BB100001000000FFFFFFFF000000000000000028
:10BB200059062014032145012882003241003219B0
:10BB300000411300390300B506002D03002D02005B
:10BB40002201002201003E01002000008009EE4D8C
:10BB50005048504F80096E4F58E5854F80096E4F11
:10BB6000B867C14F5048D04FB867C14FE828DF4F82
:10BB70008009EE4F18EAFC4F8009EE4F58E505505A
:10BB8000A4550D50F0C51450A4550D5000002110BF
:10BB9000422063308440A550C660E7700881299137
:10BBA0004AA16BB18CC1ADD1CEE1EFF131121002DF
:10BBB00073325222B5529442F772D6623993188387
:10BBC0007BB35AA3BDD39CC3FFF3DEE362244334AB
:10BBD00020040114E664C774A44485546AA54BB5D7
:10BBE00028850995EEE5CFF5ACC58DD5533672267F
:10BBF00011163006D776F6669556B4465BB77AA727
:10BC000019973887DFF7FEE79DD7BCC7C448E558CA
:10BC10008668A7784008611802282338CCC9EDD976
:10BC20008EE9AFF9488969990AA92BB9F55AD44A1E
:10BC3000B77A966A711A500A333A122AFDDBDCCBC6
:10BC4000BFFB9EEB799B588B3BBB1AABA66C877CEA
:10BC5000E44CC55C222C033C600C411CAEED8FFD16
:10BC6000ECCDCDDD2AAD0BBD688D499D977EB66EBE
:10BC7000D55EF44E133E322E511E700E9FFFBEEF66
:10BC8000DDDFFCCF1BBF3AAF599F788F8891A98128
:10BC9000CAB1EBA10CD12DC14EF16FE18010A10012
:10BCA000C230E3200450254046706760B983989302
:10BCB000FBA3DAB33DC31CD37FE35EF3B102901262
:10BCC000F322D2323542145277625672EAB5CBA5CE
:10BCD000A89589856EF54FE52CD50DC5E234C324B2
:10BCE000A01481046674476424540544DBA7FAB7A2
:10BCF0009987B8975FE77EF71DC73CD7D326F23602
:10BD00009106B01657667676154634564CD96DC9ED
:10BD10000EF92FE9C899E9898AB9ABA94458654851
:10BD200006782768C018E1088238A3287DCB5CDB41
:10BD30003FEB1EFBF98BD89BBBAB9ABB754A545AA1
:10BD4000376A167AF10AD01AB32A923A2EFD0FED0D
:10BD50006CDD4DCDAABD8BADE89DC98D267C076CF1
:10BD6000645C454CA23C832CE01CC10C1FEF3EFFE1
:10BD70005DCF7CDF9BAFBABFD98FF89F176E367E41
:10BD8000554E745E932EB23ED10EF01E30313233DA
:10BD90003435363738394142434445461000400077
:10BDA00080000001000200040008001010001800CC
:10BDB000200030004000600080000001FFFFFFFF16
:10BDC00001FF01FFFF0101FFFF0100000000000073
:10BDD0000000000000000000000000000000000063
:10BDE000020000000000000014000000020000003B
:10BDF0000700000002000000020000000000000038
:10BE0000020000000000000014000000020000001A
:10BE1000010000000200000002000000020000001B
:10BE2000000000001400000000000000FFFFFFFF02
:10BE3000FFFFFF01FFFF01FFFF01FF01FF01FFFF08
:10BE4000FF0101FFFFFF01FF0101FFFF000100FFF4
:10BE5000010000FF000064009E00C800E80002012D
:10BE600019012C013D014C015A01660172017D014D
:10BE7000870190019901A101A901B001B701BE019B
:10BE8000C401CA01D001D601DB01E101E601EB01E9
:10BE9000EF01F401F801FD010102050209020D02A2
:10BEA0001102140218021B021F022202250228029C
:10BEB0002B022E023102340237023A023D023F02C7
:10BEC0004202450247024A024C024F02510253020B
:10BED000560258025A025C025F0261026302650266
:10BEE000670269026B026D026F02710273027502D2
:10BEF000760278027A027C027E027F02810283024D
:10BF000084028602880289028B028C028E028F02D2
:10BF10009102920294029502970298029A029B0261
:10BF20009D029E029F02A102A202A302A502A602F6
:10BF3000A702A902AA02AB02AD02AE02AF02B00292
:10BF4000B102B302B402B502B602B702B902BA0234
:10BF5000BB02BC0200000000000000000200000064
:10BF600004000000001003EB0000000001000000CE
:10BF70000100000004000000000100320000000089
:10BF800000000000000000000100000001000005AA
:10BF900000000000000000000000000001000000A0
:10BFA000010000350000000001000000000000005A
:10BFB000040000000000002000000000010000005C
:10BFC0000000000004000000000000D80000000095
:10BFD0000100000000000000010000000000000659
:10BFE000000000000100000000000000010000004F
:10BFF000020000010000000000000000000000003E
:10C00000010000000300009F00000000010000008C
:10C010000000000001000000000000B90000000066
:10C02000010000000000000001000000000000AB63
:10C03000000100FF010000FF000100FF010000FF00
:10C04000FF00000100FF00010001000000FF00FFF1
:10C0500000FF00000100FFFF00FF010000000001E1
:10C06000010000FFFFFF01FF0101000000000101CE
:10C0700000030201000005020100000103010000AD
:10C08000030301000100030100010203010002009B
:10C090000301000202030100030203010003040381
:10C0A0000100040203010000000302000003030278
:10C0B0000000060302000100030200010303020066
:10C0C000010603020002010302000204030200024F
:10C0D0000703020003030302000001070300000638
:10C0E0000703000100040300010007030001040727
:10C0F000030001070703000200070300020407030F
:10C1000000020707030003020703000306070300FA
:10C1100004020703000406070300050104030005E9
:10C1200002070300050607030006000703000604D4
:10C1300007030006070703000703070300070707B5
:10C1400003000802070300080607030009020703AB
:10C150000009060703000A020703000A0707030095
:10C160000B050703000C030703000C070703000D72
:10C17000070703000E070703000E060704000E075B
:10C180000704030E070704030E070704030E07073F
:10C1900004030E070704030E070704030E07070432
:10C1A0000300070002020100000202000401020273
:10C1B0000007010202020200020201010102020163
:10C1C0000601020203050002020402000202020646
:10C1D000010202030001020203050102020503003D
:10C1E0000202040501020202040202020207020224
:10C1F0000205030102020506010202060001020215
:10C200000603010202020503020202060302020102
:10C2100006040202010607020202030402020203EC
:10C2200007020202060702020302070202030507D1
:10C2300002020307070202040704020205010402C6
:10C2400002050107020205030702020506070202B2
:10C25000060207020206050702020701070202079B
:10C26000040702020801040202080207020208058C
:10C27000070202090304020209040702020A000776
:10C2800002020A020702020A050702020A0707025F
:10C29000020B030702020B060702020C010702024F
:10C2A0000C040702020D010702020E000702020E33
:10C2B000040702020F010702020F050702020E0423
:10C2C0000703030F030703030F070703030F070702
:10C2D000030300000002020000000202000000024E
:10C2E0000200000002020000000202000000020240
:10C2F0000001000202000400020200070002020125
:10C30000010002020104000202010700020202030E
:10C3100000020201040102020106010202030500FB
:10C3200002020204010202030101020203030102EC
:10C3300002040101020204040102020206020202D6
:10C3400003020202020106030202020203020201C8
:10C3500002070202010407020203030302020204AD
:10C360000402020205070202030107020203050498
:10C370000202040107020204030702020506030287
:10C380000205000702020502070202050407020275
:10C39000060007020206020702020605070202065D
:10C3A0000707020207040702020707040202080245
:10C3B0000702020805070202090107020209040731
:10C3C00002020A000702020A030702020A06070223
:10C3D000020B020702020B050702020C0107020210
:10C3E0000C050702020D020702020C010703030CF1
:10C3F000060703030D020703030E020703030E07DC
:10C400000703030000000202000000020200000017
:10C41000020200000002020003000202010000020A
:10C4200002010200020200050102020202000202F1
:10C4300003010002020201010202020401020201E0
:10C4400002020202010402020203040102020202C9
:10C4500002020202050202020002070202000407B1
:10C46000020200060702020102070202010407029B
:10C470000201060702020203070202020507020286
:10C480000302070202030407020204020702020475
:10C49000040702020406070202050107020205035F
:10C4A0000702020505070202060207020206040748
:10C4B0000202060607020207040702020801070239
:10C4C000020900070202090107020209030702022A
:10C4D0000A000702020A020702020B000702020B0F
:10C4E000020702020C000702020B060702020C04FC
:10C4F0000702020C060702020D030702030C0007E5
:10C5000003030C020703030C050703030C070703CF
:10C51000030D050703030D070703030D07070303B7
:10C520000D070703030D070703030D070703030D9B
:10C53000070703030E0D0B07696E636C7564652FA7
:10C54000647269766572732F6D6B5F6164632E63CD
:10C5500000696E636C7564652F64726976657273C9
:10C560002F6D6B5F6165732E630033324B206C6FF0
:10C570006164206361702076616C2025640D0A007F
:10C580005854414C206C6F61642063617020766167
:10C590006C2025640D0A00556E65787065637465BE
:10C5A0006420646D61206368616E6E656C0D0A00C5
:10C5B000696E636C7564652F647269766572732F3A
:10C5C0006D6B5F666C6173682E630052656C6F61A2
:10C5D000642076616C756520696D706F7373696234
:10C5E0006C650D0A00696E636C7564652F64726911
:10C5F000766572732F6D6B5F6D6973632E63007365
:10C6000079735F7469636B5F7374617274005265F0
:10C6100073657420627920756E6B6E6F776E207310
:10C620006F757263650D0A0025313064207C200D22
:10C630000A00437261736865642121210D0A002D8F
:10C640002D2D2D2D2D2D2D2D2D2D2D2D2D2D2D2D1A
:10C650002D2D2D2D2D2D2D2D2D2D2D2D2D2D2D2D0A
:10C660002D2D2D2D2D2D2D0D0A00253038583A2039
:10C670002530385820253038582025303858202586
:10C680003038580D0A005052494D41534B3D25302A
:10C6900038580D0A00434F4E54524F4C3D25303808
:10C6A000580D0A004D53503D253038580D0A0050A2
:10C6B00053503D253038580D0A0041495243523DF0
:10C6C000253038580D0A004C523D253038580D0A97
:10C6D00000495053523D253038580D0A00785053C8
:10C6E000523D253038580D0A004E3D25642C205A05
:10C6F0003D25642C20433D25642C20563D25640DAA
:10C700000A0046494C45202020203A20005B534334
:10C710005030335D005B464952415D005B555742E6
:10C720005D005B4D41435D005B4343435D005B56F1
:10C730004552424F53455D005B53455D005B554399
:10C74000495D005B5741524E5D005B494E464F5D6F
:10C75000005B4150505D005B4552524F525D005BA3
:10C760004F535D005B424F4F545D005B5445535443
:10C770005D005B4452565D005B5048595D00696E38
:10C78000636C7564652F647269766572732F6D6B67
:10C790005F74726163652E6300257300696E636C5C
:10C7A0007564652F647269766572732F6D6B5F7542
:10C7B0006172742E6300556E65787065637465648C
:10C7C000207561727420256420737461746520255E
:10C7D0006400556E657870656374656420646D618E
:10C7E000206368616E6E656C202564005061726123
:10C7F0006D74657220696E76616C69640075617232
:10C80000745F646D615F63616C6C6261636B007522
:10C810006172745F626175645F736574004F706507
:10C820006E20414E5425640D0A00B9CCBCFEB0E622
:10C83000B1BE3A5557422DB1EAC7A9205625642EFC
:10C8400025642E200D0A00C9E8B1B849443A2025D4
:10C8500078202E0D0A006C73705F7363616C655FE6
:10C86000663332006C73705F675F6F705F66333280
:10C87000006C73705F675F6F705F696E7431360054
:10C880006C73705F675F6F705F696E7438002E2E17
:10C890002F2E2E2F2E2E2F2E2E2F2E2E2F647269FE
:10C8A000766572732F6D6B5F6C73702E63004F70C3
:10C8B0006572616E642061646472657373202578AB
:10C8C00020697320696E76616C6964004E656564E9
:10C8D000206174206C65617374206F6E65206F70C9
:10C8E0006572616E64005258204445534320696E5E
:10C8F000646578206973206F7665722072616E6757
:10C90000650D0A00455420696E64657820697320BE
:10C910006F7665722072616E67650D0A002E2E2F8C
:10C920002E2E2F2E2E2F2E2E2F2E2E2F6472697626
:10C930006572732F6D6B5F6D61632E63006D616354
:10C940005F72785F646573635F636F6E7374727533
:10C950006374006D61635F65745F636F6E7374729F
:10C9600075637400556E646566696E6564206269FE
:10C9700074207261746520256420666F72206D6575
:10C98000616E20505246206F662025640D0A004DCE
:10C9900045414E2050524620706172616D6574654C
:10C9A00072206572726F720D0A00436F64652069B0
:10C9B000647820256420616E64206D65616E20506E
:10C9C000524620256420636F6E666C6963740D0A9D
:10C9D000002E2E2F2E2E2F2E2E2F2E2E2F2E2E2FA0
:10C9E000647269766572732F6D6B5F7068792E6300
:10C9F0000001000001000000FF00FFFF0000FFFF3A
:10CA000001000100010000FF01FF01010001000021
:10CA100000000101FF000000010000FF0000FFFF17
:10CA200000FF01000100FFFF00FF01010100010103
:10CA300000000001FF00010000FF000101FF0001F4
:10CA400001010000FF01000001000100FF000101E1
:10CA5000FF01FFFF010000000000000100000000D6
:10CA600000FF0100000000FF00FF000000FFFF01C9
:10CA7000010100000100FF010000010000010000B1
:10CA800000000000FF000000FF0000FFFF000000AA
:10CA9000FF0001FF0100FF0001FF00FF0100000097
:10CAA000000001FF0000010100FF00010000FFFF86
:10CAB0000100000101FF010001FF00010000000072
:10CAC000FF00FF00FF00FF0101FF01000100000166
:10CAD0000001000000FF0100010101000000FFFF54
:10CAE000FFFF0101010000000001010100FFFFFF45
:10CAF00001FF00000000010000FFFF000000000037
:10CB0000FF000100010001FF000100000100000121
:10CB100000FF0000FF010101000001000000FF0113
:10CB2000000100FF000000000101010101FF010000
:10CB300001FFFF0001FF000101FFFF00FF000000F7
:10CB40000100FF010000010001FFFFFFFF000000E6
:10CB5000FF000000000000FF01000001FF000101D4
:10CB60000000000101FF00000101FF00FF00FF01C4
:10CB7000000101000000000000FF000100FF0100B3
:10CB8000FFFFFF01FF01010000FF010001010001A3
:10CB900000010001000000FF0000FF0000FF010095
:10CBA0000001FF0101000000FF01FF00FF01010083
:10CBB000FF000101010100FF0000FF000101000072
:10CBC00001000100000101FF00000100000001FF61
:10CBD000000000FF00FFFF0100000000FF00000058
:10CBE00000FFFF0001000000000001FFFF01000046
:10CBF00000FFFF00000000FFFF010100FF01010135
:10CC00000100FF000101000100FF0000FF01000121
:10CC10000100000101FF0001010001FF0100FF0010
:10CC200000010000FF00FFFF000000FF01FF000007
:10CC30000100000000FF000101FF000000000001F2
:10CC4000FF00FF000000000000FF0000FF01FF01E7
:10CC500001FF01000000FF0001000100010101FFD0
:10CC60000000FFFF000001000100000001000000C3
:10CC7000010100FF000100FF000001FF00FF0100B3
:10CC8000FF000001000100000000010001FF0000A2
:10CC900000000101000001000101010101FF01008C
:10CCA000FF0001FF00FFFF01000101FFFF00000086
:10CCB000FFFFFF000100000001000100FF01FF0075
:10CCC000000000000001FF01FF00FFFF0000010164
:10CCD000000000FF00000100000101FF0000FFFF55
:10CCE0000101FF0000FF00000000000001FF000044
:10CCF0000100FF000000FF010100000000FFFFFF36
:10CD00000101000000010001FF00FF010000FF0120
:10CD1000000000FFFF00FF0000FFFF00FFFF010118
:10CD200001FF0100FF0101000001FF0101000100FE
:10CD3000000000000100FF00010101FF00000100F0
:10CD40000001000000FF00000000010000FFFF01E3
:10CD50000001010001000100FF0000FF00FF01FFD2
:10CD600000010001010000000000010100000000BE
:10CD70000100000001000001FFFF0001FF010100B0
:10CD8000FF000000FFFF000001FF000100000101A3
:10CD9000000000010101000001000100FF00FF018F
:10CDA000FF00FF0001000001000001000101FFFF82
:10CDB000FFFF0100000101FFFF010001FF00FFFF75
:10CDC00001000000000000FF00FF00000000FF0164
:10CDD00000FFFF000001000000000001FF01010052
:10CDE0000000FF00FF0100010001FFFF000000FF45
:10CDF00000FF0000000001FF000000000001000033
:10CE00000000000001FFFF01FF010100FF00010021
:10CE100001000001FF000001010100FF010100FF0E
:10CE200000000100FF01000000010100010101FFFD
:10CE300000FFFF00010001FF00FFFF0000FF0000F6
:10CE400001000000FF01010000000001000101FFDE
:10CE500001FF00000100010001FFFF0000FFFF00D3
:10CE6000FF00000001000001FFFF000101010000C0
:10CE70000000010101FFFFFFFF00000001010100B0
:10CE800001FF0000000100010000010001FF01019D
:10CE9000FF00FF00FF00FF000000000100FF010095
:10CEA00001FF0101000001FFFF00000100FF000180
:10CEB000010000FF01000000000001FF00FF010071
:10CEC000FF0001FF0100FF000000FFFF0000FF0066
:10CED0000000FF0000000000000100000100000150
:10CEE000FF000100000101FF00FF01010000FF0140
:10CEF00001000000010100FF01000001FF0000002F
:10CF0000000000FF000000FFFFFFFF010001000024
:10CF100001FF0001000000FF00FFFF010100FF0111
:10CF200000FFFF010001FF010101010100000000FD
:10CF3000FF00010001FF000000010000010101FFEE
:10CF40000000FF000100000100000100FF010001DE
:10CF5000000100FF0000000000FFFF0000010000D2
:10CF60000000FF01FF00FFFF0100000000000100C2
:10CF7000FFFF00000000FF0000000001FFFF00FFB6
:10CF8000000000FF01000000010000FF010100009F
:10CF90000100010000010100FF0000FF000101018C
:10CFA0000100FF000101FF00FF01FF00000001017F
:10CFB000FF01000001FF0000FF0000FF0000000172
:10CFC000000100010001010001FF00000101FF015B
:10CFD000FFFFFF0001FF000100FF00000000000054
:10CFE00001010001FF0100010000FFFF0000FF013F
:10CFF00001010001000100FF00000001FF0101FF2D
:10D0000001FF0000FF000000000000FF00FF010022
:10D0100000000000FF010100FF000000000100000F
:10D02000FF01FF000000FFFF00FF0000010000FF04
:10D030000001FF0100010100FF01010000010100EA
:10D0400001FF0000FF000100010100FF00010101DC
:10D0500001FF000101FFFF00000000FFFF000000D2
:10D060000100000000FF0000FF0101FFFF0000FFC2
:10D0700001010000010000FF00000001010000FFAD
:10D08000FF00FF01FF01000000000000FF01FF00A2
:10D090000100010000000100FFFFFF000000FFFF92
:10D0A00001010001FFFF00FF0100FF0001FF01017E
:10D0B00001010100010000010100000000FF01006A
:10D0C00001000000000100010000FF0001FF00FF5F
:10D0D000010000FF000100FF00010100000001004D
:10D0E0000000000000000101000100FF01FF00FF3F
:10D0F0000000FF000100010001010001FFFF00002E
:10D100000100000000FF000000010000010000FF1E
:10D1100001010100FF000100000000000100010109
:10D12000FF0100000101FF0001FF010101FFFF00FD
:10D13000FFFF0000FF00FFFF00000001FF000001F3
:10D14000FF00FF0100010000000101FFFFFF0000E0
:10D1500000000101FF000000FF00010000FF0100CE
:10D160000000010001FF00FF0000000101FF0100BD
:10D1700000000000010000FFFF0001FF00000000B0
:10D18000FF00FF00000000000001FFFF00FF0100A2
:10D1900001FFFF0101000001FFFFFFFF010100018E
:10D1A00000000100000100FF00FF01FF00FF00017F
:10D1B0000001000001010100000001010000010068
:10D1C000FF010000FFFF000000FF000101FF010060
:10D1D000FFFF01000001000000010000000001014C
:10D1E00000FF000000000100FF000101010001FF3D
:10D1F00000000001FF0101010000FF0100FF00002D
:10D2000000010001FF00010001000000FF0101001A
:10D21000FF01FFFFFF00000100000101000000FF0F
:10D2200001000101000000FF01FF010100000101F8
:10D2300000010000FF00000000FF000100FF0000EF
:10D24000000001FF0000FF0000FF010101010001DB
:10D25000FF010000000100FF00010100FFFF0001CD
:10D26000FF0000010101FF01000000FF01000101BA
:10D270000100FF000100000000FF000001010000AC
:10D28000010000FFFFFF01FF000101FF000000019E
:10D29000000100FF0100010000000001000000008B
:10D2A00001FF000100010000010000000100010178
:10D2B000FFFFFF00FF010000FF0100010000FF0071
:10D2C000FF00010100000000FFFF010000FF01005E
:10D2D0000101FF010100010000FF0001010101FF48
:10D2E000FF01FFFF01FF01010101FF01FFFFFF013E
:10D2F00001FFFF010101010101FF0101FF01000028
:10D3000001FFFF0100FFFF01000101010101FFFF1B
:10D31000010101FFFF00FFFF0001FF01FFFFFFFF11
:10D3200000FF01FF01FF010001FFFF0101FF01FFFD
:10D330000101010001010001FF01FFFFFF010101E7
:10D340000101FF01FF0101FFFF01FFFF0101FFFFDD
:10D35000FF01FF0001010100FF01010101FF0100C8
:10D360000100FFFF0001FF0101FF010101010101B7
:10D37000FFFF01FF01010000010101FFFF0001FFAC
:10D38000FFFFFFFF01FF0001FF01FF01FFFFFF01A2
:10D390000101FFFF010101FFFFFF01FF01FF00FF8E
:10D3A00001FFFF000101FF01FF0100FF0101010179
:10D3B000010101010101FFFF01FFFF0101FF010167
:10D3C000000101FF01FF01FFFF01FFFF010101FF5C
:10D3D000FFFF00FF010101FF00010000FFFFFF014F
:10D3E00001FF01FFFF00FF0101000101010101FF39
:10D3F000FF010101FF0101FFFFFF01FF01FFFF002E
:10D400000101FFFFFF01FF010001FFFFFFFFFF011F
:10D4100000010101FFFF01FF01FFFF01FF0101FF0B
:10D420000101010100FF00FF0101000001FF0101F6
:10D4300001FF0101FF0100FF0100FFFF01FFFFFFEE
:10D44000010101000101FF00FFFF01FF0101FFFFDA
:10D4500000010100000101FF0101FFFFFFFFFF01CB
:10D460000101010101FF0001FFFF01FF0101FFFFB9
:10D4700001FF010101FFFF01010101010101FF01A4
:10D4800001010001FF01FF00FF00FF0101FFFFFF9D
:10D490000100FFFFFF010100FF01FF01FF0101FF8C
:10D4A000FF010100FFFF000101FF0000FFFF01017C
:10D4B000FF0101FF01FFFF0101010101FFFFFF016A
:10D4C0000101FF01FF0001FF01FF01000101010156
:10D4D00001FF010101FF010101FF0100FFFFFFFF4B
:10D4E000FFFF0101FF0101FF0100FFFFFFFF01FF3F
:10D4F00001FF00010001FF010101FFFF01FF010128
:10D5000000010101FFFF0101FF0001010000FFFF19
:10D510000101FFFF010101FF01FFFFFFFFFFFF000E
:10D52000010101FF0101010101FFFF01FF0101FFF5
:10D53000FFFF01FF01FFFFFF01FF0100FF01FFFFF0
:10D5400000010001FF0101FF01010001FF01FFFFD8
:10D55000000101010101FF010101010101010101BE
:10D560000101FFFFFF01FF0101FFFF01010000FFBB
:10D5700001FF0100FF01FF00FF0101FFFF010101A9
:10D58000FF01010100FFFF000101FF01FF01FF009A
:10D59000FFFFFF0101FF00FFFFFFFF01010101FF8E
:10D5A00001FF000100FF01FF0101FF0101FFFF0179
:10D5B000FF04000004040404040404040000000048
:10D5C000E0D500000890010220050000E40A0000F8
:10D5D000D8D7000028950102BC290000CEBA00006F
:10D5E00052033280420133010142644E03050902B5
:10D5F0000302020101010002035026E43D9A1FCA02
:10D60000C37ED3FBA84FC434EB2E360F22EB14A8F5
:10D610005060F8AA36D3D1748614140026B80301DA
:10D6200045900050084202C203001515C0C1C2C394
:10D63000C4C5C6C7C8C9CACBCCCDCECF0001010175
:10D640004301806509020301420257140019412772
:10D6500017901D0706050403020100F29798DDC824
:10D660009D5CB81CC0DEA7DB615BCA0102000352EF
:10D67000404805100406010001522D2C280004002A
:10D680007C007B0105020308FF5B0F010065F901C7
:10D69000417B0707010160002000881333E05364D9
:10D6A00020ACFF501B0D070E080E080E080E080CCC
:10D6B000030D050B050D070D070D070D0701012EC5
:10D6C000010402004003FFFF7F00FFFF7F0816FFF9
:10D6D000FFFF00FFFFFF3A010001000A0001010601
:10D6E000401E400512051200051504020102030147
:10D6F00002400402010303020C0E0900087A023200
:10D70000413428002A820303455006C570014013A6
:10D71000E620700140144C07001000D6FF00B00056
:10D72000500B4202820345FFFF0F203204420832B1
:10D7300001045510000134B40003055020005007C7
:10D740009D2800040001020100FFFFFFFF379890B1
:10D75000010203C40051151EC135BF80F3E2BDC0F4
:10D76000B464BF871699BDAD178DBF941799BD33AB
:10D77000A876BFC4780DBD2BC162BA0CB0AFBEA9EC
:10D78000F6E9BAFC567BBE07254CBBEC8823BE5D90
:10D79000C0CBBB0CCE20BD7BA095BCD40F3A3E2D98
:10D7A0005EACBD5913073F640100424209440300C7
:10D7B000063201451001400FC20E52014590014052
:10D7C000184204023D0545A00140194206023D07EA
:08D7D000454001400D820100FB
:020000040000FA
:10DB0000A5A54B4D0000001000000002AAAA5A7FF4
:10DB100000DB000000000000020000000000000028
:10DB200000000000000000000000000000000000F5
:10DB300000000000000000000000000000000000E5
:10DB400098DB0000000000000A56656E646F7209E1
:10DB50003A204D4B53454D490A43686970093A20B4
:10DB60004D4B383030300A44617465093A204A75AB
:10DB70006E20323520323032350A56657273696F45
:10DB80006E093A2056302E362E320000000000007A
:08DB900000000000000000008D
:04000005000000C136
:00000001FF
